:1000000040090020819D00002D9E00002F9E0000D1
:10001000319E0000339E0000359E0000000000006D
:10002000000000000000000000000000333B000062
:10003000379E000000000000E13A00009D3C0000F7
:10004000399E00003B9E0000A76A0000B16A0000D4
:100050003D9E00003F9E0000419E0000439E000028
:10006000459E0000479E0000DF6B0000EB6B000028
:10007000499E0000A79B00004B9E00004D9E000083
:10008000995F00004F9E0000519E00000D89000006
:10009000539E0000559E0000579E0000599E000090
:1000A0005B9E00005D9E00005F9E0000619E000060
:1000B000639E0000659E0000679E0000699E000030
:1000C0006B9E00006D9E0000119C00006F9E000062
:1000D000719E0000739E0000759E0000779E0000D8
:1000E000799E00007B9E00007D9E00007F9E0000A8
:1000F000819E0000839E0000859E0000879E000078
:10010000899E00008B9E00008D9E00008F9E000047
:10011000919E0000939E0000959E0000979E000017
:10012000999E00009B9E00009D9E00009F9E0000E7
:10013000A19E0000A39E0000A59E0000A79E0000B7
:10014000A99E0000AB9E0000AD9E0000AF9E000087
:10015000B19E0000B39E0000B59E0000B79E000057
:10016000B99E0000BB9E0000BD9E0000BF9E000027
:10017000C19E0000C39E0000C59E0000C79E0000F7
:08018000C99E0000CB9E0000A7
:10018800F8B504002089001910F10E0520890830FF
:100198002081082600273A003100280000F0ECFFF3
:1001A8002800F2BD010008894018801D0A89083A14
:1001B8000A817047010008894018801D7047521A4B
:1001C800401A92B280B2824201D3012000E000209E
:1001D800C0B27047401A00B2002801D5012000E0E3
:1001E8000020C0B2704738B504000D00210089B264
:1001F800280080B2FFF7EEFF32BD401A002801D573
:10020800012000E00020C0B2704738B504000D009E
:1002180021002800FFF7F1FF32BD2DE9F84F040057
:100228000D0016001F00DDF82880002D0AD11420CB
:1002380001F056F80500002D02D15FF0FF3079E09B
:10024800002028812800FFF79BFF8146380080B2F4
:1002580001F05CF9A9F80400404680B201F056F9B3
:10026800A9F806007010D9F8001060F38201C9F8E7
:100278000010B010D9F8001060F34101C9F800105F
:10028800D9F8000066F3C300C9F80000F010D9F8E7
:10029800001060F30001C9F80010F00717D5280016
:1002A80001F0FFF800900098002802D15FF0FF30BD
:1002B80040E001F04AF900994860002200A9206D49
:1002C80001F058F9012802D0009801F082F8E0689E
:1002D8008246E068800F012802DAE068800F00E0BB
:1002E800012060F39F7A5FEA1A5010F01F0001F0B6
:1002F80097F9834600235A462900504601F05EFAD2
:1003080000280FD0DFF8D8060078002804D0DFF8DE
:10031800701C002001F0D8FB280001F05AF87FF08B
:10032800050007E0B00704D5A4F82C8001F00DF90A
:10033800A0640020BDE8F28F2DE9FC410400642090
:1003480000F0CEFF0500002D02D15FF0FF3048E03D
:1003580000202881606D01F044F9070000200600A4
:10036800BE4236DADFF81C2C01A9606D01F02FF9C6
:1003780001280AD0DFF868060078002804D0DFF8E2
:10038800081C002001F0A0FB23E00198FFF712FFF2
:100398008046B8F8040001F0B9F82989490815EB36
:1003A8004101C8812889801C2881DFF834064079FA
:1003B800002806D0B8F80420DFF8D01B052001F08B
:1003C80083FBDFF8C02B01A9606D01F0E4F8761C0F
:1003D800C6E7208D0090638C062229002000FFF7D5
:1003E8001CFFBDE8F68111B581B00C000198406989
:1003F800002817D0002201A90198406901F0BAF835
:1004080000280CD1DFF8D8050078002804D0DFF8E0
:10041800801B002001F058FB7FF0080019E0002045
:10042800019948612000FFF7BDFE2100019801F005
:10043800E3FB00280CD5DFF8A8054078002804D095
:10044800DFF8501B012001F03FFB7FF0080000E0BF
:10045800002016BDF8B50400606D01F0C2F8060072
:1004680000200500B54242DADFF8182B00A9606DBC
:1004780001F0ADF801280AD0DFF8640500780028FB
:1004880004D0DFF8041B002001F01EFB2FE00098C9
:10049800FFF790FE0700DFF848054079002805D0EF
:1004A800BA88DFF8F41A052001F00EFBB888218D10
:1004B800491C89B2884212D1DFF824054079002806
:1004C80005D0BA88DFF8D41A052001F0FDFA0099A2
:1004D8002000FFF788FF208D401C2085BCE7DFF84F
:1004E800A42A00A9606D01F056F86D1CBAE7F1BDA9
:1004F8002DE9F04182B004000D00606D01F071F843
:10050800070000200600BE423BDADFF8782A00A97F
:10051800606D01F05CF801280AD0DFF8C4040078A7
:10052800002804D0DFF8781A002001F0CDFA28E07E
:10053800DFF8502A00A9606D01F02DF80098FFF748
:1005480039FE8046DFF898044079002806D0B8F8CC
:100558000420DFF8501A052001F0B6FAB8F80400B4
:10056800ADB2A8420BD1DFF878044079002804D056
:10057800DFF83C1A052001F0A7FA012002E0761CFA
:10058800C1E70020BDE8F68132B504001500290056
:1005980089B22000FFF7ACFF002801D0002005E059
:1005A800DFF8E02900A9606D00F0F5FF32BD2DE904
:1005B800F84F04000D00206D01F013F8804600206C
:1005C8000600464580F28380002200A9206D00F0D5
:1005D800EDFF01280AD0DFF808040078002804D0CD
:1005E800DFF8C419002001F06FFA70E00098FFF7F7
:1005F800E1FD8146DFF8E803407900280CD0B9F81E
:10060800040000F089FF03009BB200984268DFF8FD
:100618009C19052001F058FA5FF0000A0020070035
:1006280028890838B7EB500F34DA15EB4700C08932
:1006380000F072FF8346B9F8040000F06DFF1FFA5E
:100648008BFB834501D101208246B9F8040000F0F4
:1006580063FF834615EB4700C08900F05DFF1FFA72
:100668008BFB834514D200F070FF83460098016825
:100678005846FFF7CAFD00280AD0A06BBBEB000064
:10068800401E00994860A06B1BEB50000099086061
:100698007F1CC5E7BAF1000F05D1002200A9206D23
:1006A80000F068FF11E0CE48407900280AD0B9F878
:1006B800040000F031FF80B20200DFF81C1A0520A8
:1006C80001F002FA009800F084FE761C79E7BDE894
:1006D800F18F38B50400E06B002807D1A08D218D7B
:1006E800884201D001201AE0002018E000F02DFF18
:1006F8000500A06C216C09182800FFF786FD00286A
:1007080001D001200BE0A08D616C091889B2208D01
:10071800FFF769FD002801D0012000E0002032BD6C
:1007280010B582B00400002C02D0206D002809D139
:10073800AB480078002804D0DFF82819002001F021
:10074800C3F943E0DFF83C2800A9206D00F03FFF23
:10075800012819D100980028F4D0A1484079002830
:100768000ED00098FFF726FD808800F0D5FE030024
:100778009BB200984268DFF8F018052001F0A4F950
:10078800009800F026FEDDE7DFF8F82700A9606D85
:1007980000F01DFF012819D100980028F4D09048D6
:1007A800407900280ED00098FFF704FD808800F0FB
:1007B800B3FE80B2030000984268DFF824190520D0
:1007C80001F082F9009800F004FEDDE713BD70B572
:1007D80082B00400012500200600012E0EDA14EB79
:1007E8008600006900F0FDFE216BD0F164008142B3
:1007F80002DB0020050001E0761CEEE7002D0CD09E
:100808002000FFF766FF002807D0208D0090638C3A
:10081800022200212000FFF700FD002076BD2DE90F
:10082800FC47040000F091FE05006069002814D020
:10083800A069616B09182800FFF7E7FC00280CD0B5
:1008480067484078002804D0DFF89018012001F0AC
:100858003BF9200001F02BFBC0E094F920000428AC
:1008680014D1A069616B09182800FFF7CEFC002895
:100878000BD05B484079002804D0DFF868180520C1
:1008880001F022F9200001F012FBA7E0206D00F032
:10089800A8FE070000200600BE4280F28280DFF832
:1008A800CC2701A9206D00F092FE012802D1019801
:1008B800002809D14A484078002804D0DFF82818D1
:1008C800012001F001F96CE00198FFF773FC804604
:1008D800B8F8040000F020FEA18C80B2FFF77AFC83
:1008E800002816D03E48407900280ED0B8F80400F9
:1008F80000F012FE0300A08C00909BB201984268A1
:10090800DFF8E817052001F0DFF8019800F061FD35
:1009180045E001984068A16B09182800FFF775FCAD
:10092800002836D02E48407900280AD0B8F80400AC
:1009380000F0F2FD020092B2DFF8B417052001F0D2
:10094800C3F8208D00F0E2FDA8F8060000F0FDFDD8
:1009580001994860019800F0A4FD8146E068000D07
:1009680010F01F0000F05CFE824600235246494604
:10097800E06800F023FF00280BD0194840780028D1
:1009880004D0DFF87017012001F09EF8484600F007
:1009980020FDDFF8D82601A9206D00F0FCFD761CAB
:1009A8007AE72000FFF713FF94F92000032815D1F8
:1009B800206D00F016FE216B88420FDA206B80B2A2
:1009C800410089B2608CA28C801A80B2FFF702FCC9
:1009D800002803D014F14C0001F01EFBBDE8F3879A
:1009E800000000202DE9F04387B004000D00280026
:1009F800FFF7E0FB0600F08800F08EFDF080B0887D
:100A080000F08AFDB080DFF8F006407900281ED09B
:100A180028890838069028890590F0880490B088BD
:100A28000390307810F0010002903068C0F3400065
:100A380001903068C0F3800000903068C0F3C003B4
:100A480094F92020DFF8B416052001F03DF830783D
:100A5800C00756D53068C0F38000002802D0F0885F
:100A6800401CA08494F92000042803D094F92000A5
:100A7800002810D1DFF880064079002804D0DFF87C
:100A88008016052001F020F8280000F0A2FC2000C4
:100A980001F00DFA70E2DFF860064079002806D010
:100AA80094F92020DFF85C16052001F00DF8B088D5
:100AB800218D491C89B2884218D1DFF83C0640795B
:100AC800002804D0DFF84016052000F0FDFF0420C0
:100AD80084F8200000F039FDA061208D0090638C1F
:100AE8000A2200212000FFF798FB2DE2DFF8080614
:100AF8004079002804D0DFF81416052000F0E4FF40
:100B080037E294F9200000280AD0022800F0D880A3
:100B1800C0F08080042800F0CF81C0F0D18009E2C5
:100B28003068C0F3C000002812D1DFF8CC05407946
:100B3800002804D0DFF8D815052000F0C5FF208D67
:100B48000090638C082200212000FFF766FBFBE180
:100B5800DFF8A4054079002804D0DFF8B81505208F
:100B680000F0B2FF00F0F1FC01F074FA01F082FA33
:100B7800E084E08C401C6084E08CA084B0882085F0
:100B8800B0886085B088A085D5F80E0000F0D7FC45
:100B98002063D5F8120000F0D2FC6063D5F8160087
:100BA80000F0CDFCA063D5F81A0000F0C8FCE063A3
:100BB800D5F81E0000F0C3FC2064D5F8220000F030
:100BC800BEFC6064DFF830054079002808D0A06BCF
:100BD8000090636B226BDFF84015052000F074FF6E
:100BE800DFF814054079002808D0606C0090236C69
:100BF800E26BDFF82815052000F066FF022084F874
:100C08002000608D0090E38C032200212000FFF774
:100C180004FBAEE1307810F00C000C2829D1B08824
:100C28002085B0886085B088401EA085F088401C6B
:100C3800A08400F08AFCA064032084F82000DFF878
:100C4800B8044079002804D0DFF8D414052000F057
:100C58003BFFE06B002807D1208D0090638C0222B7
:100C680000212000FFF7D9FA14F14C0001F0D4F963
:100C78007FE13068C0F38000002816D0DFF87804E0
:100C88000078002804D0DFF89C14002000F01CFF36
:100C9800208D0090638C082200212000FFF7BDFA08
:100CA80014F14C0001F0B8F963E1DFF84C04007866
:100CB800002804D0DFF87014002000F005FF43E19D
:100CC800307810F00C00042819D0B088618D884263
:100CD8000AD0DFF824040078002804D0DFF84C1488
:100CE800002000F0F1FE2FE1DFF80C044079002825
:100CF80004D0DFF83C14052000F0E6FE39E1208D31
:100D0800216B10EB410292B2208D411C89B2B08850
:100D1800FFF755FA002826D1DFF8DC0340790028D0
:100D28000DD0208D401C216B10EB41000090208DD0
:100D3800431CB288DFF8FC13052000F0C5FE94F9C7
:100D48002000022807D1608D0090E38C0322002147
:100D58002000FFF762FA94F92000032802D120004E
:100D6800FFF7EAFA05E1608C421E92B2A08C401EA1
:100D7800216BB0EB410189B2F088FFF720FA002817
:100D880013D1DFF87403007800280DD0608C401E62
:100D98000090A08C401E216BB0EB4103F288DFF875
:100DA8009813002000F090FEE3E094F92000022858
:100DB8001BD1F088E18C88420AD0DFF83C03007828
:100DC800002804D0DFF87413002000F07DFEBBE09B
:100DD800DFF824034079002804D0DFF864130520E5
:100DE80000F072FE032084F82000F088401CA084E4
:100DF8003068C0F34000002807D02889092803D3A9
:100E080029002000FFF7D3FBB3E028890928C0F0A8
:100E1800B080B088218D491C89B2884215D0B2882B
:100E280029002000FFF7B0FB01280AD0DFF8C8022C
:100E38004079002804D0DFF80C13052000F044FEA8
:100E480097E02000FFF778FA96E0B788290020009D
:100E5800FFF7C9FA002840F08C802785D5F80A00EA
:100E6800800F01000020804614EB8800006900F024
:100E7800B8FB8146206B10EB090065280DD22000D5
:100E8800FFF727FC002813D0208D0090638C0222E6
:100E980000212000FFF7C1F90AE0DFF85C02407981
:100EA800002805D0228DDFF8A012052000F00CFEE6
:100EB8002000FFF7CFFA5FE0307810F00C0004282C
:100EC8000AD0DFF834024079002804D0DFF87C1219
:100ED800052000F0F9FD4CE0608C421E92B2A08C17
:100EE800401E216BB0EB410189B2F088FFF767F92A
:100EF800002813D1DFF80002007800280DD0608C9C
:100F0800401E0090A08C401E216BB0EB4103F2887C
:100F1800DFF82412002000F0D7FD2AE0F088401CFA
:100F2800A084208D0090638C0A2200212000FFF706
:100F380074F91EE0DFF8C0010078002804D0DFF85B
:100F48001012002000F0C0FD606900280ED1DFF803
:100F5800A8014079002804D0DFF8F811052000F036
:100F6800B3FD0021200000F047FE02E0200000F061
:100F78009EFF280000F02DFA07B0BDE8F0830000BE
:100F880008AB000088000020D0A600002CB40000A8
:100F980018A8000040B4000044A80000C8B400002D
:100FA80000A7000070A800009CA8000030AB00005B
:100FB800D8B4000010B504004F48C078002804D009
:100FC80022006549032000F07FFD002084F82000FE
:100FD80062480068606362480068A06314F14C00CE
:100FE80000F0DDFF01280AD043480078002803D02C
:100FF8005C49002000F068FD5FF0FF3031E004211B
:10100800142000F0A8FA2065206D00280ED13A4877
:101018000078002803D05449002000F055FD14F151
:101028004C0000F0CFFF5FF0FF301AE004212820C9
:1010380000F091FA6065606D002811D12E480078A3
:10104800002803D04949002000F03EFD14F14C006F
:1010580000F0B8FF206D00F087FA5FF0FF3000E085
:10106800002010BD58AB000004AE0000880000202E
:1010780010B582B0040094F92000002801D10020A6
:1010880029E094F92000042819D0042084F82000CD
:1010980000F05BFAA061208D0090638C0A22002189
:1010A8002000FFF7BAF814484079002804D022003D
:1010B8002F49052000F008FD7FF00B000BE00E48DB
:1010C8004079002803D02B49052000F0FDFC0020C2
:1010D80084F82000002016BD54B4000080AB000046
:1010E80028AE000068B4000030A70000C8A80000BF
:1010F800F4A8000040B3000000000020B09F0000EA
:10110800B4A3000058B3000074A4000020A9000094
:101118006CA600007CB4000024A50000B0A4000068
:10112800F0B10000A8AB000044B000004CAE0000D5
:1011380064B000005CA5000060A700000CB20000CD
:1011480028B2000044B200002CA3000070AE0000DA
:1011580060B2000084B00000D0AB00008000002026
:1011680084000020A4B0000094AE0000B8AE0000D7
:10117800C4B00000F8AB000062F30F2262F31F4214
:10118800401810F0030308D0C91A1FD3DB0748BF63
:1011980000F8012D28BF20F8022D130030B41446A2
:1011A8001546103928BF20E93C00FAD8490728BF5E
:1011B80020E90C0048BF40F8042D890028BF20F81A
:1011C800022D48BF00F8012D30BC7047C91818BF60
:1011D80000F8012DCB0728BF00F8012D704700004B
:1011E8002DE9F04782B004000D00B948046015F1FC
:1011F8001200B8490860B748006810F10807F81CE1
:1012080080088700B248006807FB00F8404600F0F5
:10121800A1FFB1490860B0480068002834D0042113
:10122800AB48006800F097F9AC490860AB48006823
:10123800002804D1A848006800F092FF24E05FF07D
:101248000009A548D0F800A04A4641465046FFF795
:1012580093FF002006009E480068864212D29E48EE
:10126800006807FB060000900020009908600098BD
:1012780000994860002200A99848006800F07AF9AF
:10128800761CE8E7002001E05FF0FF30BDE8F68754
:101298001CB5040000200090002001908D480068D3
:1012A80014F11201884201D2002018E001AA00A915
:1012B8008A48006800F08BF90098002801D10020C6
:1012C8000DE0009800994968884201D0002006E0A6
:1012D80000980068401C009908600098083016BD06
:1012E80010B582B00400002000907A48006814F11C
:1012F800120188420AD27A480078002804D02200D5
:101308007849002000F0E0FB002033E0002200A92B
:101318007248006800F04AF90098002809D170481E
:101328000078002803D07049002000F0CDFB002091
:1013380020E06B48C078002806D000984368009ADF
:101348006A49032000F0C0FB009800994968884268
:1013580009D063480078002803D06549002000F0D0
:10136800B3FB002006E000980068401C0099086064
:101378000098083016BD1CB5040000200190002C10
:1013880026D0B4F10800009000980421B0FBF1F2D7
:1013980002FB1102002A1BD100984068009988427C
:1013A80016D100980068002812D00098006802281A
:1013B80005D300980068401E0099086008E00020E6
:1013C8000099086001AA00A94448006800F0E3F801
:1013D80013BD10B582B00400002C08D14048007835
:1013E800002803D04349002000F06EFB58E0B4F118
:1013F8000800009000980421B0FBF1F202FB1102F2
:10140800002A09D036480078002804D022003A493A
:10141800002000F059FB43E000984068009988429A
:1014280009D02F480078002804D022003349002032
:1014380000F04AFB34E000980068002809D12848E9
:101448000078002804D0009A2D49002000F03CFBC9
:1014580026E000980068022810D300980068401E13
:10146800009908601E480078002806D00098036894
:10147800009A2449002000F027FB11E00020009981
:1014880008601748C078002804D0009A1E49032035
:1014980000F01AFB002200A91048006800F06AF862
:1014A80013BDF8B504002500002D01D100200DE082
:1014B8002889FFF715FF0600002E06D005480768A3
:1014C8003A002900300000F051FE3000F2BD000063
:1014D80018DC00201CDC002014DC002010DC0020BC
:1014E8000000002078A90000B8B4000018B500007A
:1014F800A0B3000024AF0000A0A90000C0AC000009
:1015080044AF0000E4AC000024B5000080B2010242
:1015180051EA102080B2704710B50400200080B254
:10152800FFF7F4FF10BD010651EA106110F47F4285
:1015380051EA0221000A10F47F400843704710B5B1
:1015480004002000FFF7EFFF10BD80B501F031F86F
:101558000521484302BD38B504000D0000222900CA
:10156800200001F037FC32BD10B50400200001F066
:10157800A7FE10BD70B504000D00160016F1010F8E
:1015880002D00520B6FBF0F6002332002900200027
:1015980001F083FC70BD70B504000D001600002337
:1015A80032002900200001F018FD70BD70B504005C
:1015B8000D00160016F1010F02D00520B6FBF0F65B
:1015C800002332002900200001F068FD70BD70B5CD
:1015D80004000D00160032002900200001F010FE62
:1015E80070BD10B50400200001F05BFE10BD0000C6
:1015F80001002E48C9B2052202FB0100006800283C
:1016080005D02A48C9B2052202FB010007E0274895
:10161800D0F8A000002801D0254800E0002070473D
:1016280010B504002000C0B2FFF7E2FF0100002956
:1016380001D1002000E0086810BD10B504002000AA
:10164800C0B2FFF7D5FF0100002901D1FF2000E05B
:10165800087910BDF8B504000D0016001F00002E13
:1016680002D17FF001001FE0300001F0EFFEE4B28C
:10167800212C0DDA0D48E4B2052101FB04000660B7
:101688000A48E4B2052101FB0400077100200BE0C1
:1016980008480078002805D0E4B222000649002056
:1016A80000F012FA7FF00100F2BD000014D800200B
:1016B800B4D800200000002020AC0000DFF8801320
:1016C80008707047DFF878030078704738B5040071
:1016D8002000C0B2FFF7F2FF00F0C3FA0500002DAA
:1016E80001D0280022E001F0EBFE0500002D01D01A
:1016F80028001BE001F03CFF0500002D01D0280068
:1017080014E0DFF8400301F0A1FEFFF7DBFFFF2341
:10171800DFF830230521C0B2FFF79CFFFF23DFF875
:10172800242305212020FFF795FF002032BD38B57E
:101738000400E0060BD5DFF810030078002804D079
:10174800DFF80813002000F0BFF9002035E060073B
:101758000BD5DFF8F4020078002804D0DFF8F01287
:10176800002000F0B1F9002027E0DFF8E802044289
:101778000BD0DFF8D4020078002804D0DFF8D812A4
:10178800002000F0A1F9002017E0012000F029FB5B
:101798000500002D01D100200FE0E00509D5042146
:1017A8006420FFF7D8FE68616869002803D100202B
:1017B80003E000206861EC61280032BD2DE9F043A8
:1017C80087B006000F0090469946002F0AD1DFF82F
:1017D80078020078002804D0DFF88012002000F09A
:1017E80073F98DE0B8F1000F03D0D8F8080000288D
:1017F8000BD1DFF854020078002805D03200DFF85A
:101808006012002000F060F97AE0DFF83C0200790D
:10181800002817D0D8F80000059038890490F0B255
:101828000390B00F0290C6F305200190C6F38530EF
:101838000090C6F30453C6F34462DFF8281204206C
:1018480000F042F9C7F80A60FFF73CFFC6F34461AD
:10185800C9B2C0B281422FD1300000070AD5DFF8E3
:10186800E8014078002804D0DFF8FC11012000F0DE
:101878002BF940E03000C00710D50021380001F0F6
:1018880023FF00280AD0DFF8C0014078002804D0E0
:10189800DFF8D811012000F017F92CE030004007DC
:1018A8000AD5DFF8A4014078002804D0DFF8C01179
:1018B800012000F009F91EE03C89B8F80C50ADB2DF
:1018C800002D03D0ADB2A4B2A54214D34A463900C4
:1018D8004046D8F80830984700280CD1D8F81000AE
:1018E800401CC8F81000D8F82C00A4B22018C8F87A
:1018F8002C00002006E0D8F81800401CC8F8180092
:101908007FF0090007B0BDE8F08338B504000D008A
:10191800002C02D0E069C00501D4002007E00020B7
:1019280000902A0000A96069FFF740FE009832BDC8
:101938002DE9F84F04000D0016001F00DDF828807F
:10194800DDF82C90DDF830A0D9F80A00000A000272
:10195800C9F80A005FEAC8700AD53B480078002831
:1019680003D04449002000F0AFF87FF0010063E0A5
:101978005FEA48700AD534480078002803D03E4909
:10198800002000F0A1F87FF0040055E05FEAC8608D
:101998000AD52D480078002803D03849002000F0E7
:1019A80093F87FF0040047E05FEA486005D5D9F86E
:1019B8000A0050F00100C9F80A00EDB2D9F80A008F
:1019C80065F31850C9F80A00F6B2D9F80A0066F3A8
:1019D8009330C9F80A00FFF775FEC0B2D9F80A10AB
:1019E80060F35D61C9F80A10FFB2D9F80A0067F31D
:1019F8000D20C9F80A00E4B2D9F80A0064F39F7010
:101A0800C9F80A002800C0B2FFF70AFE8346002082
:101A180010EB0901897A00AA8154401C0428F7D3E5
:101A280053465A4649460098FFF7C8FE002802D098
:101A38007FF0040000E00020BDE8F28F0000000005
:101A4800D8DC00204400002000000020D4A00000C2
:101A58002CA10000AAFEFFFFF8B20000B8AA0000FF
:101A680010B3000074A3000014A0000028B3000005
:101A78004C9F0000ECA4000084A1000034A20000E8
:101A8800FEB504000D0016001F00002C02D17FF0E7
:101A9800010017E0029701950096D4F80A00800B20
:101AA80010F03F03D4F80A00000A10F03F02D4F8FF
:101AB8000A00400E10F01F01D4F80A00800FC0B2CF
:101AC800FFF736FFFEBD00000CB4F8B504000D00AA
:101AD800F02664B2072C04DA344864B2205C00288B
:101AE80000D13EE064B2002C0CD0022C07D00CD3FD
:101AF800042C10D00CD3062C13D00FD314E01320D1
:101B0800060012E0122006000FE0142006000CE088
:101B18000620060009E00320060006E0052006006E
:101B280003E00720060000E01BE006A807001E48A7
:101B38000068002807D03A002900200040B21A4B5C
:101B48001B6898470DE03000C0B201F021FE390053
:101B5800280001F071FE13A001F07AFEF02001F0D8
:101B680017FEF1BC5DF80CFB10B5040064B2072C3D
:101B780003DB0F4801F06CFE12E00C4864B2205CF5
:101B8800002801D0002000E00120084964B2605418
:101B9800064864B2225C64B22100064801F058FE8F
:101BA80010BD00000D0A000028DC00200000002005
:101BB800C8B30000E0B2000010B5002004000A2CF1
:101BC80019DADFF88403582101FB040090F90100B9
:101BD80001280ED1DFF87003582101FB0400007AB8
:101BE800800706D5DFF86003582101FB0400FEF7E3
:101BF80016FE641CE3E710BD32B50400002C02D1C8
:101C08007FF001002CE00098002807D00098D0F859
:101C18000A00800F01000020050001E000200500F7
:101C2800002200A914EB85000069FFF7A3FC012836
:101C380015D0DFF81803007800280DD014EB8500C4
:101C48000069FFF7CEFC030014EB85000269DFF89A
:101C580000130020FFF738FF5FF0FF3000E000209E
:101C680032BD70B5FFF771FC00F0F4F900F002FA2C
:101C7800202190FBF1F202FB110212F12000DFF8A3
:101C8800D4120870DFF8D00200F089F901280CD0CE
:101C9800DFF8B8020078002804D0DFF8C01200206E
:101CA800FFF712FF5FF0FF305FE0002004000A2C0E
:101CB80047DA00200500012D0DDADFF88C025821E3
:101CC80001FB040010EB850604216420FFF743FCA8
:101CD80030616D1CEFE70020DFF86C12582202FB20
:101CE80004114870DFF86002582101FB0400001D50
:101CF80000F048F901280CD0DFF8500200780028DD
:101D080004D0DFF85C120020FFF7DEFE5FF0FF3042
:101D18002BE0DFF83402582101FB0400FFF74AF9F1
:101D280000280CD0DFF824020078002804D0DFF85F
:101D380034120020FFF7C8FE5FF0FF3015E0641C86
:101D4800B5E7DFF8240200F02AF901280CD0DFF803
:101D5800FC010078002804D0DFF810120020FFF7FB
:101D6800B3FE5FF0FF3000E0002070BD30B4020029
:101D7800002003000A2B17DADFF8CC01582505FBF1
:101D88000300040094F9010000280BD094F9000026
:101D9800002807D1A068084011EA0205A84201D12D
:101DA800200002E05B1CE5E7002030BC704738B536
:101DB800040000200500012D11DA002200A914EB0F
:101DC80085000069FFF7F2FB012806D1009800287A
:101DD800F3D00098FFF7FDFAEFE76D1CEBE7002062
:101DE80032BDF8B504006421DFF87C0100F0F6F894
:101DF80001280BD0DFF854010078002804D0DFF860
:101E080070110020FFF760FE00203CE0DFF864015D
:101E180000780700781C0A2190FBF1F201FB1207F9
:101E2800002005000A2D11DADFF81C01582101FBFA
:101E38000700060096F90100002807D0781C0A213F
:101E480090FBF1F201FB12076D1CEBE796F901001C
:101E580001280DD13D480078002804D0DFF818117A
:101E68000020FFF731FE404800F0D6F800200AE0D5
:101E7800012070700020706134703E4807703A4845
:101E880000F0CAF83000F2BD70B504000D00002063
:101E9800FFF7A7FF0600002E07D0B460F560FFF734
:101EA80054FBB0613000FFF782FF300070BD10B501
:101EB8000400002C0AD125480078002803D02F49B7
:101EC8000020FFF701FE7FF001003BE094F90100DC
:101ED800002809D11D484079002803D02849052049
:101EE800FFF7F2FD00202DE0207A800702D4207B46
:101EF800800707D52000FFF7BBF810F10C0F01D1C0
:101F080000201FE06421184800F068F801280AD072
:101F18000E480078002803D015490020FFF7D4FDAB
:101F28007FF002000EE0002060702000FFF73FFF06
:101F3800207A800702D52000FEF7F2FB0A4800F05D
:101F48006BF8002010BD0000CCD10020000000205C
:101F580064AF0000D6DC002024DC002008AD0000BF
:101F68002CAD000004A6000020DC002050AD0000CD
:101F780064B10000D7DC002080B1000084AF00000D
:101F8800B4B3000010B50400012000F058FF206031
:101F98002068002801D0012000E0002010BD10B505
:101FA800040003220021012000F014FF20602068B3
:101FB800002805D0002300220021206800F06DFFD2
:101FC800012010BD10B50400002C05D020680028A1
:101FD80002D02068FFF7C8FA012010BD38B5040008
:101FE8000D0019488079002804D0220017490620DE
:101FF800FFF76AFD15F1010F02D00520B5FBF0F5DA
:1020080000232A000021206801F048F8012801D1A6
:10201800012000E0002032BD10B504000A48807994
:10202800002804D022000A490620FFF74DFD0023AE
:1020380000220021206800F030FF012801D1012092
:1020480000E0002010BD00000000002030B50000B6
:102058003CB5000010B504460448C046C0460021FF
:1020680001700348C046C046046010BD4009002006
:1020780044090020F8B5344F3846C046C0460446E7
:10208800381DC046C046054607F10800C046C04690
:10209800064607F10C00C046C04623782B492C4A57
:1020A800002B40D12B6802FB03132B60082702FB8F
:1020B80003132B6002FB03132B6002FB03132B603B
:1020C80002FB03132B6002FB03132B6002FB0313B9
:1020D8002B6002FB03132B600346D5F800C002FBFC
:1020E8000C1CC5F800C043F804CB7F1ED5F800C00F
:1020F80002FB0C1CC5F800C043F804CBD5F800C09F
:1021080002FB0C1CC5F800C043F804CBD5F800C08E
:1021180002FB0C1CC5F800C043F804CBDDD1C36F2B
:102128003360012323702B6802FB03112960317887
:1021380001F01F0150F8212032602A6840F8212060
:10214800306880008008F2BD400900205FF36E3CD3
:102158000D66190010B50400200001F08BFB10BDBE
:1021680010B50400200001F007FC10BD62B38B0716
:1021780008D0521E11F8013B00F8013B00F0248002
:102188008B07F6D1830740F0208000BF103A07D3B1
:1021980030B4B1E83810103AA0E83810F9D230BCA1
:1021A800530724BFB1E80810A0E8081044BF51F84D
:1021B800043B40F8043BD20724BF31F8022B20F837
:1021C800022B44BF0B7803707047083A07D3B1E875
:1021D8000810083A40F8043B40F804CBF7D25307FC
:1021E800E4E700002DE9FA4F83B0040015000E9EC5
:1021F8000F9FDDF84080DDF844902000002802D1D0
:1022080001F089FCFEE7072E02D301F084FCFEE70B
:102218004146280080B200F077FC8246BAF1000FF0
:1022280075D0DAF83000ADB210EB8500001F834698
:102238005FEADB0B5FEACB0B1BF00700002802D03C
:1022480001F069FCFEE7280080B200904B4632009E
:102258000399504600F094FB049A2100584601F077
:1022680085FCCAF80000002F01D0C7F800A001F0D3
:10227800E4FCDFF8B8050068401CDFF8B01508601A
:10228800DFF83806006800280BD1DFF83006C0F800
:1022980000A0DFF898050068012811D100F0A8FB1C
:1022A8000EE0DFF808060068002809D1DFF80C0600
:1022B8000068C06A864203D3DFF80006C0F800A0B1
:1022C800DFF8EC050068401CDFF8E4150860DFF86B
:1022D800E0050068CAF84000DFF8D8050068012169
:1022E800DAF82C2091400843DFF8C81508601AF185
:1022F8000401DFF8C405DAF82C20142303FB0200DC
:1023080001F027FD0120019001F0AFFC02E05FF031
:10231800FF300190019801280CD1DFF89005006882
:10232800002807D0DFF894050068C06AB04201D2DF
:1023380001F07AFC019805B0BDE8F08F2DE9F8436B
:1023480004000D005FF00008002C02D101F0E3FB4F
:10235800FEE7002D02D101F0DEFBFEE7DFF8A00763
:102368000068002802D001F0D6FBFEE700F0A5F8CF
:10237800DFF80806D0F800902068281806002068C2
:10238800814507D2206886420BD2B14509D2012087
:10239800804606E02068864201D3B14501D201207B
:1023A80080462660B8F1000F19D0DFF810050068E4
:1023B800001D01F0F7FC00280ED1DFF800050068C9
:1023C800DFF8F01409680122C06A12FA00F031EA55
:1023D8000000DFF8E0140860300000F06BFB00F04C
:1023E80074F80700002F01D101F01EFCBDE8F1834D
:1023F80070B504000026002C2BD0DFF80407006815
:10240800002802D001F087FBFEE700F056F8DFF85D
:102418006C05006820180500DFF8A0040068001D9E
:1024280001F0C0FC00280ED1DFF890040068DFF846
:10243800841409680122C06A12FA00F031EA000027
:10244800DFF870140860280000F034FB00F03DF855
:102458000600002E01D101F0E7FB70BD1FB500207A
:10246800039000200290002001900020009000239B
:102478004FF48072DFF878180FF2E540FFF7B2FEEC
:102488000400012C13D101F046FB5FF0FF30DFF8A8
:10249800641808600120DFF8141408600020DFF8D1
:1024A800DC14086001F092FC01F07AFB04E0002CD7
:1024B80002D101F030FBFEE71FBDDFF844060068DB
:1024C800401CDFF83C160860704738B50025DFF877
:1024D800E0050068002802D101F01DFBFEE701F0CD
:1024E800ACFBDFF8CC050068401EDFF8C4150860B7
:1024F800DFF8BC050068002857D1DFF83003006812
:10250800002852D0DFF8E407006800282AD0DFF856
:10251800DC07C068C068040014F1180001F042FC30
:10252800201D01F03FFCDFF88C0300680121E26AFE
:1025380091400843DFF87C130860211DDFF8780319
:10254800E26A142303FB020001F003FCE06ADFF8EF
:102558006C130968C96A8842D4D30120DFF8C4170C
:102568000860CFE7DFF890070068002814D0DFF88C
:102578008807006800280FD000F020F8002803D052
:102588000120DFF8A0170860DFF86C070068401E1C
:10259800DFF864170860EAE7DFF8880700680128B1
:1025A80003D10120050001F03FFB01F05EFB28008C
:1025B80032BDDFF8C8130968080070472DE9F041FB
:1025C8000026DFF8EC04006800287AD1DFF8AC03B5
:1025D8000068401CDFF8A4130860DFF8A003076850
:1025E800002F1FD1DFF8340700680068002802D0E8
:1025F80001F091FAFEE7DFF8240700688046DFF86B
:1026080020070068DFF814170860DFF81407C0F81F
:102618000080DFF814070068401CDFF80C1708601A
:1026280000F0A8FADFF8CC06006887423CD3DFF850
:10263800EC0600680068002805D15FF0FF30DFF87D
:10264800B416086030E0DFF8D4060068C068C068D7
:10265800040060680500AF4203D2DFF89806056001
:1026680022E0201D01F09EFBA06A002803D014F18F
:10267800180001F097FB8F4800680121E26A914039
:1026880008438C490860211D8B48E26A142303FB28
:10269800020001F05EFBE06A88490968C96A88425D
:1026A800C5D301200600C2E7834884490968C96A7E
:1026B800142202FB01000068022809D30120060049
:1026C80006E0DFF834060068401CDFF82C160860C6
:1026D800DFF850060068002801D00120060030000D
:1026E800BDE8F08138B5DFF8C8030068002804D0D9
:1026F8000120DFF83016086062E00020DFF82416B9
:10270800086001F073FBDFF824160860DFF8200684
:102718000068DFF81816096888420BD26748006815
:10272800016DDFF8082612685118DFF804261268D0
:10273800891A0165DFF8F4050068DFF8F415086008
:102748005E480068006B05005FF0A530040028684B
:10275800A04208D16868A04205D1A868A04202D169
:10276800E868A04207D05548006810F13401534882
:10277800006801F06DFB4F480068B0FA80F0D0F1B6
:102788001F0004004C48142101FB040000680028C5
:1027980002D101F0C0F9FEE74749142202FB0411F7
:1027A8000800416849684160416810F10802914297
:1027B80002D14168496841604068C0683F49086083
:1027C80031BD70B504000D00002C02D101F0A3F951
:1027D800FEE73A48006810F11801200001F0C5FA38
:1027E80036480068001D01F0DDFA00280BD1334897
:1027F8000068304909680122C06A12FA00F031EA1B
:1028080000002C49086015F1010F07D12B4800681A
:10281800011DDFF8F00201F09CFA06E05748006855
:1028280028180600300000F045F970BD98DC00203B
:1028380070B50400E068C0680500002D02D101F001
:102848006AF9FEE715F1180001F0ACFA984800683B
:10285800002813D1281D01F0A5FA164800680121A7
:10286800EA6A9140084313490860291D1248EA6A38
:10287800142303FB020001F06CFA05E015F11801BE
:10288800DFF8680401F065FA0C480068C06AE96A74
:10289800884206D2012006000120DFF8981408605B
:1028A80001E000200600300070BD0000A4DC00201C
:1028B800B4DC0020A0DC0020BCD8002088DC00208C
:1028C80010B50400002C02D101F025F9FEE7DFF86D
:1028D800580400682060DFF860040068606010BD7C
:1028E800F8B504000D00002C02D101F014F9FEE740
:1028F800002D02D101F00FF9FEE701F09EF91F4803
:102908000768286810F1010F02D1002006001DE0B9
:10291800DFF8140400682168884205D0606887429F
:1029280002D30120060011E06068381A296888423D
:102938000AD22868C01B6168081828602000FFF7C1
:10294800BFFF0020060001E00120060001F08DF91C
:102958003000F2BD0120DFF8DC130860704700008A
:1029680010B5040000F070F8DFF8D40300680228FE
:1029780001D301F059F9C046C046F3E79CDC0020BA
:102988002DE9F04104000D0016001F0000208046CC
:10299800B8F10A0F0CD218F8050018EB040181F8F9
:1029A800340018F90500002802D018F10108EFE7F3
:1029B800002084F83D00072E01D306200600E662B9
:1029C800A6640020E064201D0021016114F11800B4
:1029D800002101612461D6F10700A0616462002032
:1029E800206500206065002084F85800BDE8F0816B
:1029F80010B500200400072C08D2DFF84403142186
:102A080001FB040001F096F9641CF4E7DFF83403D5
:102A180001F090F9DFF8300301F08CF9DFF8CC020F
:102A280001F088F9DFF8240301F084F9354801F052
:102A380081F9DFF81003DFF8E4120860DFF8080313
:102A4800DFF8DC12086010BD38B5DFF80403006851
:102A580000282BD0FFF731FDDFF8F00200680028CE
:102A680001D1012400E00024FFF72FFD002CECD158
:102A780001F0E3F8DFF8D402C068C0680500281D3B
:102A880001F090F9DFF8CC020068401EDFF8C412AC
:102A98000860DFF8BC020068401EDFF8B412086066
:102AA80001F0E3F8280000F05CF8CEE731BD000043
:102AB800BCDC002010B50400DFF89C02006844600C
:102AC800DFF874020068844209D2DFF88C020068DB
:102AD800011DDFF84C02006801F047F90EE0DFF84D
:102AE80078020068011DDFF83402006801F03DF942
:102AF80080480068844201D27E48046010BD00000E
:102B0800BCDC0020C8DB00202DE9F84304000D00E0
:102B1800002D04D1A4B2A00000F0ACFE00E0280013
:102B28000700002F0BD05C2000F0A4FE0600002E4A
:102B380001D0376305E0380000F01EFF01E00020F7
:102B48000600002E0AD0A4B2A7005FF0A508D6F8A8
:102B58003090424639004846FEF70EFB3000BDE88B
:102B6800F28310B50400206B00F006FF200000F08F
:102B780003FF10BD694909680968002904D15FF09D
:102B8800FF315C4A116007E064490968C968C9688F
:102B980008004168574A1160704738B5040025009D
:102BA800002C4FD0E86ADFF8B0110968C96A88427A
:102BB80048D2A869002806D4DFF89C010068C06ADA
:102BC800D0F10700A8616869DFF87411EA6A142374
:102BD80003FB0211884230D1281D01F0E3F80028D8
:102BE80012D1DFF85C01E96A142202FB01000068D7
:102BF800002809D1DFF8440100680121EA6A914000
:102C08008843DFF838110860DFF84C010068C06AB3
:102C1800E862DFF8280100680121EA6A9140084368
:102C2800DFF818110860291DDFF81401EA6A142377
:102C380003FB020001F08DF804E0DFF81C010068D6
:102C4800C06AE86231BD70B5040025000026002C7A
:102C58004AD0DFF804010068854202D000F05BFF2B
:102C6800FEE7E86C002802D100F055FFFEE7E86CAB
:102C7800401EE864E86AA96C884235D0E86C0028F0
:102C880032D1281D01F08EF8002812D1DFF8B000EB
:102C9800E96A142202FB01000068002809D1DFF864
:102CA8009C0000680121EA6A91408843DFF88C1093
:102CB8000860A86CE862E86AD0F10700A861DFF84C
:102CC8007C0000680121EA6A91400843DFF86C1033
:102CD8000860291DDFF86800EA6A142303FB020074
:102CE80001F037F801200600300070BDA0DB00209D
:102CF800A8B50000B8DC0020A8DC0020DFF85800E8
:102D08000068002805D0DFF850000068C16C491C35
:102D1800C164DFF844000068704700008CDC0020C4
:102D280090DC0020ACDC0020B0DC0020C4DC0020FB
:102D3800C0DC0020ACDC00209CDC0020A0DC0020F3
:102D4800BCD8002078DB00208CDB0020B4DB00201E
:102D580094DC002098DC002088DC002070B504009A
:102D68000D002600002E02D100F0D5FEFEE700F08F
:102D780064FF3068F16B326C02FB01007060002068
:102D8800B0633068B0603068F16B491E326C02FB8A
:102D98000100F0605FF0FF3070645FF0FF30B064F6
:102DA800002D0BD13069002810D016F11000FFF764
:102DB8003FFD01280AD100F037FF07E016F11000A7
:102DC80000F0B8FF16F1240000F0B4FF00F04DFF4A
:102DD800012070BD2DE9F84304000D0016005FF0D6
:102DE8000009002C02D100F096FEFEE7002D02D16A
:102DF8000020804603E005FB04F0401C804618F1E3
:102E0800540000F037FD0700002F0FD0002D01D12E
:102E18003F6002E017F154003860FC633D64012113
:102E28003800FFF79BFF87F85060B946B9F1000FEB
:102E380002D100F070FEFEE74846BDE8F28338B5DF
:102E48000400542000F016FD0500002D23D00020BA
:102E58006860002028600020A8600020E86000204A
:102E6800A8630120E863002028645FF0FF306864ED
:102E78005FF0FF30A86485F8504015F1100000F0AD
:102E880059FF15F1240000F055FF0023002200210E
:102E9800280000F002F8280032BD2DE9F7430400AD
:102EA8000D001E005FF00008A146B9F1000F02D125
:102EB80000F031FEFEE7002D03D1D9F840000028CC
:102EC80001D1012000E00020C0B2002802D100F0AA
:102ED80022FEFEE7022E03D1D9F83C00012801D1D9
:102EE800012000E00020C0B2002802D100F013FE4B
:102EF800FEE700F0A2FED9F83800D9F83C10884265
:102F080001D3022E1AD132002900484600F0E4F914
:102F18000700D9F82400002808D019F12400FFF789
:102F280087FC012806D100F07FFE03E0002F01D0C6
:102F380000F07AFE00F099FE01204CE0029800288B
:102F480003D100F092FE002045E0B8F1000F04D153
:102F580000A8FFF7B5FC0120804600F086FEFFF7C9
:102F6800ACFA00F06AFED9F8440010F1010F02D162
:102F78000020C9F84400D9F8480010F1010F02D127
:102F88000020C9F8480000F070FE02A900A8FFF769
:102F9800A7FC002819D1484600F047FA00280ED0AF
:102FA800029919F11000FFF70CFC484600F0F8F9F7
:102FB800FFF78BFA00289CD100F036FE99E74846C7
:102FC80000F0EEF9FFF781FA93E7484600F0E8F9D8
:102FD800FFF77BFA0020BDE8FE832DE9F0470400E7
:102FE8000D0016001F00A246BAF1000F02D100F032
:102FF80092FDFEE7002D03D1DAF84000002801D148
:10300800012000E00020C0B2002802D100F083FDBA
:10301800FEE7022F03D1DAF83C00012801D1012094
:1030280000E00020C0B2002802D100F074FDFEE7E5
:1030380000F04CFE00F06FFD8146DAF83800DAF84F
:103048003C10884201D3022F20D13A002900504673
:1030580000F042F9DAF8480010F1010F0ED1DAF861
:10306800240000280FD01AF12400FFF7E1FB002804
:1030780009D0002E07D00120306004E0DAF84800BB
:10308800401CCAF848000120804601E00020804624
:10309800484680F311884046BDE8F0872DE9F7439C
:1030A80004000D001E000027A146B9F1000F02D14F
:1030B80000F031FDFEE7002D03D1D9F840000028CB
:1030C80001D1012000E00020C0B2002802D100F0A8
:1030D80022FDFEE700F0B1FDD9F83800002834D011
:1030E800D9F80C0080462900484600F041F9002E26
:1030F80019D1D9F83800401EC9F83800D9F80000AD
:10310800002803D1FFF7FAFDC9F80400D9F8100028
:10311800002816D019F11000FFF78AFB012810D1FA
:1031280000F082FD0DE0C9F80C80D9F824000028D1
:1031380007D019F12400FFF77BFB002801D000F02D
:1031480073FD00F092FD012058E00298002803D199
:1031580000F08BFD002051E0002F04D100A8FFF7FC
:10316800AFFB0120070000F080FDFFF7A6F900F093
:1031780064FDD9F8440010F1010F02D10020C9F80C
:103188004400D9F8480010F1010F02D10020C9F815
:10319800480000F06AFD02A900A8FFF7A1FB00287B
:1031A80026D1484600F031F900281BD0D9F8000094
:1031B800002807D100F041FDD9F80400FFF7EDFC25
:1031C80000F053FD029919F12400FFF7FAFA484676
:1031D80000F0E6F8FFF779F900287FF47BAF00F0FC
:1031E80023FD77E7484600F0DBF8FFF76EF971E753
:1031F800484600F0D5F8FFF768F90020BDE8FE83DF
:103208002DE9F84304000D001600A146B9F1000F9E
:1032180002D100F080FCFEE7002D03D1D9F8400070
:10322800002801D1012000E00020C0B2002802D10E
:1032380000F071FCFEE700F049FD00F06CFC8046F0
:10324800D9F83800002824D02900484600F090F822
:10325800D9F83800401EC9F83800D9F8440010F1F0
:10326800010F0ED1D9F8100000280FD019F1100065
:10327800FFF7DEFA002809D0002E07D001203060C1
:1032880004E0D9F84400401CC9F8440001200700B4
:1032980001E000200700404680F311883800BDE8AF
:1032A800F28338B50400002C02D100F034FCFEE7AC
:1032B80000F0C3FCA06B050000F0D7FC280032BD6D
:1032C80038B504002500002D02D100F024FCFEE7EB
:1032D800280000F051FB31BD2DE9F84304000D0032
:1032E80016000027206C002809D12068002839D151
:1032F8006068FFF7A8FC07000020606032E0002E3D
:1033080013D1D4F84080D4F80890424629004846A2
:10331800FEF72CFFA068216C0818A060A0686168FF
:1033280088421FD32068A0601CE0D4F84080D4F8FD
:103338000C90424629004846FEF718FFE068216CC9
:10334800401AE060E0682168884203D26068216C16
:10335800401AE060022E05D1A06B002802D0A06BB5
:10336800401EA063A06B401CA0633800BDE8F28338
:10337800F8B504000D00206C002810D0E068216C1E
:103388000818E060E0686168884201D32068E0605E
:10339800266CE768320039002800FEF7E7FEF1BD29
:1033A80010B5040000F049FCA06C01280EDB606A2F
:1033B80000280BD014F12400FFF73AFA002801D0B6
:1033C800FFF7C8FAA06C401EA064EDE75FF0FF307D
:1033D800A06400F04AFC00F030FC606C01280EDBB1
:1033E800206900280BD014F11000FFF721FA0028FB
:1033F80001D0FFF7AFFA606C401E6064EDE75FF044
:10340800FF30606400F031FC10BD38B5040000F0F6
:1034180014FCA06B002802D10120050001E0002067
:10342800050000F022FC280032BD38B5040000F089
:1034380004FCA06BE16B884202D10120050001E089
:103448000020050000F011FC280032BD0D49096874
:10345800002904D10B4908600021816310E0094963
:103468000968814204D08A6B002A01D0896BF8E789
:10347800814205D08A6B002A02D1886300228263C8
:103488007047000044DC002001000022202901D3FD
:10349800002014E0314810F93100012805D12F48E7
:1034A80010EBC1004068020008E02C4890F90001C8
:1034B800012803D12948D0F8040102001000704700
:1034C80070B54FF484740025244E2A002100300082
:1034D800FDF752FE002070BD38B504000D00002C29
:1034E80002D17FF0010037E0EDB2212D0BDB1C4843
:1034F8000078002804D020221A490020FEF7E4FAB8
:103508007FF0010028E01548EDB210F935000028D9
:103518000CD013480078002805D0EDB22A001249D3
:103528000020FEF7D1FA7FF0030015E00C48807800
:10353800002806D0EDB22B0022000C490220FEF72D
:10354800C3FA0648EDB210EBC500446001200349F8
:10355800EDB201F83500002032BD00003CD5002056
:1035680000000020DCA20000D4B1000024B000005C
:1035780010B500200400012C15DA414850F8240049
:1035880000280ED108210A20FDF7E5FF3C4941F843
:1035980024003B4850F82400002802D15FF0FF3097
:1035A80002E0641CE7E7002010BD10B504006422A7
:1035B800210033480068FDF7F9FF012802D07FF0A9
:1035C800020000E0002010BD2DE9FC4104000D00C0
:1035D8001600002C08D12B484078002803D02A492F
:1035E8000120FEF771FA48E0002D11D125484078F6
:1035F800002803D025490120FEF766FA002E03D1E2
:103608002000FDF7E6FE02E02000FDF7B4FE34E0FE
:10361800009501945FF00008002E08D1002200A94F
:10362800174850F82800FDF7A5FF070007E032000B
:1036380000A9134850F82800FDF7ADFF0700012F37
:1036480014D010484078002803D011490120FEF713
:103658003BFA286A401C2862002E03D12000FDF79F
:10366800B8FE0AE02000FDF786FE06E06869401C07
:103678006861286B218908182863BDE8F381000078
:1036880048DC002000000020E0AA0000ECA70000B1
:1036980038A6000010B402005FF0FF3318000B00DA
:1036A800591E002B09D0074B14784440E4B253F854
:1036B800243093EA1020521CF1E75FF0FF335840A2
:1036C80010BC7047489100002DE9F04182B0040019
:1036D8000D00002C02D17FF0010023E0EDB2002D97
:1036E80007D02089011D14F10A00FFF7D3FF0090CD
:1036F80005E0218914F10E00FFF7CCFF0090009837
:10370800FDF711FF0090042600AF2089001910F181
:103718000E08320039004046FEF728FD2089001DBA
:1037280020810020BDE8F68138B504000D00002C8A
:1037380002D17FF001002AE02089042802D27FF01C
:10374800010024E0EDB2002D06D0218914F10A0011
:10375800FFF7A0FF009006E02089011F14F10E007A
:10376800FFF798FF00900098FDF7DDFE0090042217
:1037780000A9208900190A3000F074FB002802D043
:103788007FF0010003E02089001F2081002032BD66
:1037980070B50400E4B214F00F00C0B201280CD0D8
:1037A80023D303280FD00BD3052812D00ED3072814
:1037B80015D011D3082815D017E01E20050016E0F3
:1037C8001F20050013E02020050010E0212005003F
:1037D8000DE0222005000AE02320050007E0242050
:1037E800050004E02520050001E000200500E4B202
:1037F80014F0F000C0B2102806D0202807D03028D6
:1038080008D0402809D00BE0012006000AE0022079
:10381800060007E00320060004E00420060001E09B
:10382800002006002A003100024800F011F870BD9F
:103838000000000048B5000002B5024600AB0121B7
:1038480002487844801D00F03FFB02BD357B000034
:103858000EB400B582B003A90091024600AB012165
:10386800034878440A3000F02FFB06BC5DF810FBD3
:10387800117B00002DE9F04104005FF00008FEF71D
:103888001CFE8E480068002801D100F0ADF88C4875
:10389800006804425FD1002C10D08A4800680419DF
:1038A80014F0070F0AD014F1080014F00701441AA5
:1038B80014F0070F02D000F02EF9FEE7002C4AD0D2
:1038C80081480068A04246D3804806007F480068C7
:1038D80005006868A04205D22868002802D02E009A
:1038E8002D68F6E775480068854234D03068754918
:1038F80009680818804628683060724800684000E7
:103908006968091B88420FD26019070017F0070081
:10391800002802D000F0FFF8FEE76868001B786016
:103928006C60380000F097F8674800686968401ACA
:10393800654908606448006865490968884203D297
:10394800614800686249086068685D490968084319
:10395800686000202860FEF7B8FDB8F1000F01D1BB
:1039680000F07CFA18F00700002802D000F0D3F825
:10397800FEE74046BDE8F08170B504002600002C43
:103988002BD050480068361A350068684C490968D9
:10399800084202D100F0BFF8FEE72868002802D0EC
:1039A80000F0B9F8FEE7686845490968084214D08C
:1039B8002868002811D16868414909688843686007
:1039C800FEF77BFD40480068696808183E490860B2
:1039D800280000F040F8FEF778FD70BD3A4800680E
:1039E80070473B480068704730B44FF44843394C3F
:1039F800220012F0070F05D0D21DD208D2009B1A60
:103A0800344CE3181100314C216000242F4D6C60B8
:103A18005C1822002B4C2468121BD208D200274CB9
:103A280022600024254D2D686C600024234D2D68EC
:103A38002C600800141A4460204C24680460446810
:103A4800234D2C604468204D2C605FF000441C4DD1
:103A58002C6030BC704710B41C4B1A0013688342AA
:103A680001D21268FAE7110053685B18834204D147
:103A780053684468E31853601000010043685B18FA
:103A88001468A34211D113680C4C2468A34208D0CF
:103A9800436814686468E318436013681B6803602C
:103AA80005E0064B1B68036001E01368036082426F
:103AB80000D0106010BC70470000000050DC0020EF
:103AC8005CDC0020D0B5000054DC0020ECDB0020DA
:103AD80058DC0020CC090020EFF30980BFF36F8F7A
:103AE800204B1A6820E9F00F106008B54FF0A000CD
:103AF80080F31188FEF7F6FD4FF0000080F311887F
:103B0800BDE8084019680868B0E8F00F80F3098834
:103B1800BFF36F8F7047EFF311804FF0A00181F36F
:103B28001188704780F3118870470E4B1968086830
:103B3800B0E8F00F80F30988BFF36F8F4FF00000F3
:103B480080F311884EF00D0E704707480068006832
:103B580080F3088862B661B6BFF34F8FBFF36F8FEB
:103B680000DF000088DC002008ED00E0001F5FF0A7
:103B780080730360001F0160001F0FF20D030360D4
:103B8800143802602038704780B55F48006810F12B
:103B9800010F02D0FFF7BFFFFEE7FFF7BCFFFEE70C
:103BA80000B583B0594801780191FF21017001786F
:103BB8008DF800109DF8001011F0A001544A117002
:103BC8000721544A11609DF8001009060AD5514989
:103BD8000968491E4F4A11609DF8001049008DF888
:103BE8000010F0E74B49096809024A4A116049493F
:103BF800096811F4E061474A11600199017046486B
:103C0800006850F47000444908604348006850F068
:103C180070404149086000F04CF800203A490860BB
:103C2800FFF793FF00200EBD5FF080503B4908600E
:103C3800BFF34F8FBFF36F8F704780B5FFF76BFFF0
:103C480031480068401C30490860BFF34F8FBFF30C
:103C58006F8F2D480068012806D13048006800069B
:103C680002D0FFF758FFFEE701BD80B5264800687F
:103C7800002802D1FFF74FFFFEE723480068401EE7
:103C88002149086020480068002802D1002080F3FC
:103C9800118801BD80B5FFF73EFFFEF78FFC0028B5
:103CA80003D05FF080501D490860002080F3118820
:103CB80001BD1B480068C821B0FBF1F0401E19493E
:103CC80008600720184908607047000038B5EFF30E
:103CD80005800400102C0BD314480068205C0500F4
:103CE8000B480078EDB2854202D2FFF714FFFEE7D9
:103CF800084800680E49096811F4E061884202D258
:103D0800FFF709FFFEE731BD1C01002000E400E0D9
:103D1800DDDC00207CDC002020ED00E004ED00E08C
:103D28002001002014E000E010E000E0DCB5000015
:103D38000CED00E010F1080141605FF0FF31816097
:103D480010F10801C16010F1080101610021016052
:103D5800704742684A6093688B60936859609160C5
:103D6800086103685B1C0360704710B40B6813F1AB
:103D7800010F02D10469220008E010F108042200B2
:103D880054682468A34201D35268F9E754684C6028
:103D98004C68A1608A60516008610468641C046012
:103DA80010BC7047010008698A684B689A604A68C5
:103DB8008B685A6042688A4201D18A684260002250
:103DC8000A610268521E026000687047194800685C
:103DD80050F080701749086000201749086017489C
:103DE800006850F0010015490860704712490968D9
:103DF800080013490968884204D212490968491C15
:103E0800104A11600E4908600F4909680F4A91422B
:103E180007D2400B0B4909685FF4002202FB01003E
:103E280006E0800B074909685FF4802202FB010065
:103E380070470000FCED00E0041000E0001000E016
:103E480080DC002084DC002020010020801D2C0460
:103E580038B504000D00FFF75EFEFEE780B5FFF7FA
:103E68005AFEFEE70300002013F0030F09D0521E8C
:103E780022BF13F8010B11F801CBB0EB0C00F3D003
:103E88007047121F22BF53F8040B51F804CB60454A
:103E9800F7D0121D0AD200BA9CFA8CFCB0EB0C00C9
:103EA80038BF6FF0000088BF01207047521E22BF44
:103EB80013F8010B11F801CBB0EB0C00F6D0521C33
:103EC80008BF1046704700002DE9F04FA1B08046AA
:103ED800002017461D4602910B900DF1440A6FF021
:103EE80000490AE017F8011B0298C0470028029011
:103EF80000F0AB820B98401C0B90387808B90B98EF
:103F0800A5E22528EED1002005900690079008909C
:103F180009900A9001E040F0010017F8011F2029DC
:103F2800F9D023290DD02B2904D02D2906D03029EA
:103F38000AD00CE040F0020080B2EEE740F0040046
:103F4800FAE740F00800F7E740F01000F4E72A2904
:103F58000ED12968296051F8042B2960002A0D9296
:103F680004D5514240F004000D9180B27F1C11E04D
:103F780000210D9109E00D99494505D001EB810318
:103F880002EB430130390D917F1C3A78A2F13001E0
:103F98000A29F0D339782E2903D04FF0FF310C913C
:103FA8001DE017F8011F2A2907D1296829607F1CFD
:103FB80051F8042B29600C9211E000210C9109E0C2
:103FC8000C99494505D001EB810302EB43013039D7
:103FD8000C917F1C3A78A2F130010A29F0D3ADF890
:103FE80038000FF67840397800F046FE08B117F827
:103FF800010B8DF83A009DF83A00682802BF39781D
:104008006829622005D06C2804BF38786C2803D151
:1040180071208DF83A007F1C11A8049017F8014B05
:10402800B4F1250029D01C3800F0C280001F0228F6
:1040380040F2BE80133800F0E380093800F0B88001
:10404800801E00F04A81401E00F02381401E022895
:1040580040F2AE80001F00F01C81401F79D0401E46
:1040680000F0CE80401E24D0C01E0BD0801E00F071
:10407800C780C01E00F0C48039E125208DF84400B7
:1040880001203DE12868286050F8046B28600396F9
:104098000C9C002C04D5304600F0FAFD044606E0DE
:1040A80022460021304600F00FFE00B1841B069422
:1040B80027E1296829603C2451F8040B2960002174
:1040C800CDE9000111A80390DDE90001049E11B9B2
:1040D80008B90C9AB2B10206120FA0EB02123032E4
:1040E800D2B2631E3A2AA8BF2732000940EA0170FB
:1040F80009099A5508BF00281C4603D0039AA3193A
:104108009A42E8D3A0190390C4F13C010C98069197
:10411800814209DA401A08904FF6EF71BDF838006D
:104128000840ADF83800ECE0002840F1EA809DF83E
:10413800380000F01400102840F0E3800D98059A2C
:10414800801A089A801A441A012CC0F2DA8008945E
:10415800D7E09DF83A0062281AD0682806D06A2865
:104168000CD06C281CD0712808D019E02868286069
:1041780050F8041B28600B980880C2E02868286063
:1041880050F8042B28600B98C117C2E90001B8E069
:104198002868286050F8041B28600B980870B0E065
:1041A8002868286050F8041B28600B980860A8E06D
:1041B8002868C01D20F007022A60D2E900010832F1
:1041C8002A60CDE90001002902D505982D210AE0D1
:1041D800BDF83800810702D505982B2103E0C007F8
:1041E80005D50598202100F80A10401C059011A853
:1041F800059908180390214600A800F0E5F980E029
:104208009DF83A006C280DD0712818BF6A2809D18A
:104218002868C01D20F007022A60D2E90001083290
:104228002A6005E02968296051F8040B29600021FB
:10423800CDE900019DF83A00682803D1DDE90001C5
:1042480080B20BE0622803D1DDE90001C0B205E0CD
:10425800742818BF7A2804D1DDE900010021CDE9CE
:1042680000019DF8380000072ED5DDE9000100297E
:1042780008BF002828D044F02000782824D10598C9
:10428800302100F80A10401C411C059100F80A4032
:104298001AE09DF83A00294600F0DCF8CDE9000163
:1042A800002902DA05982D210AE0BDF838008107B7
:1042B80002D505982B2103E0C00705D505982021D4
:1042C80000F80A10401C059011A8059908180390D9
:1042D800214600A800F0F5F813E0012005902868B1
:1042E800286050F8041B28608DF8441009E0252048
:1042F8008DF84400012005901CB18AF80140022085
:1043080005900D980599401A0899401A0699401A7F
:104318000999401A0799401A0A99441A9DF83800D1
:10432800400710D420208DF84000002609E0012322
:1043380010AA00A9404600F07AFC002840F08580C9
:10434800761CA642F3DB059E0DF1440B0AE01BF830
:10435800011B0298C0470028029076D00B98401C99
:104368000B90761E002EF2D130208DF840004FF0D1
:10437800000B089E09E0012310AA00A9404600F09E
:1043880056FC002861D10BF1010BB345F3DB069E07
:10439800DDF80CB00AE01BF8011B0298C0470028A2
:1043A800029052D00B98401C0B90761E002EF2D132
:1043B80030208DF840004FF0000B099E09E00123E2
:1043C80010AA00A9404600F032FC00283DD10BF1AC
:1043D800010BB345F3DB03980699079E01EB000B2D
:1043E80009E01BF8011B0298C047029068B30B98BC
:1043F800401C0B90761E002EF3D130208DF8400023
:104408004FF0000B0A9E08E0012310AA00A94046BD
:1044180000F00DFCC8B90BF1010BB345F4DB9DF8B6
:10442800380040077FF569AD20208DF84000002650
:1044380000E0761CA642BFF660AD012310AA00A9D1
:10444800404600F0F4FB0028F3D04FF0FF3021B0D5
:10445800BDE8F08F622826D068281DD06A2808D0C9
:104468006C2827D0712804D0742823D07A280CD03F
:1044780020E00868C01D20F007000860D0E900238C
:10448800083008601946104670470A680A6052F8F2
:10449800040B0A60002170470A680A6052F8040B8E
:1044A8000A6000B20BE00A680A6052F8040B0A605E
:1044B80040B204E00A680A6052F8040B0A60C117A7
:1044C80070472DE9FA4E05460A462F696F2A08BF3C
:1044D800082405D041F02000782814BF0A241024AD
:1044E8003C26D5E90001642A18BF692A81468A4614
:1044F80005D1002903DAD9F100096AEB4A0ABAF1B1
:10450800000F08BFB9F1000F0CD1286B50B9082C67
:1045180036D195F83800000732D530203B2687F889
:104528003B002DE0E31748465146224600F0F8FBD1
:10453800A4FB0023A9EB02023032D2B2A6F1010B90
:104548003A2A5E4603DB9DF80030513B9A188146B3
:104558005FEA010A0BF8072008BFB9F1000F03D082
:10456800E868F1198842DDD3082C09D195F838009C
:10457800000705D5F05D302802D0761E3020F055B2
:10458800C6F13C00A861F119E960296B884208DA94
:10459800081A28624FF6EF71288F08402887BDE86F
:1045A800F38E00290ED595F8381001F01401102962
:1045B80008D1696B6A69891A2A6A891A0E1A012E42
:1045C800A8BF2E62BDE8F38E2DE9F24F04468EB0E7
:1045D800D4E90001CDE9020104AF9DF8380040F0AC
:1045E800200BBBF1610F0AD0206B002848BF0620C2
:1045F80004D408BFBBF1670F01D1012020636168B3
:10460800C1F30A5040F2FF7290421CD1080304BF64
:104618002068002809D10320A0619DF8380061387E
:104628001A2836D30FF2486108E00320A0619DF8EC
:10463800380061381A2829D30FF22C61E068032268
:10464800FDF794FDBEE1012816DA204600F0DFFBF5
:10465800012811DB00250020BBF1610F20D1E168A2
:10466800302201F8012B4A1CE2609DF83820612AAB
:104678000CBF782258220FE0626840F2FE3161F3E5
:104688001E52451A62604FF0FF30E5E70FF2D45131
:10469800D4E70FF2D851D1E70A706169891C6161CA
:1046A80010B90026002584E1BBF1610F40F0978026
:1046B800206BD4E900AB00284CBF2126461CDDE95D
:1046C80002010022002300F0C3FB36B23ABF8BF090
:1046D8000040CDE902A0CDE902AB06F101082D1F8B
:1046E8008DF810200DF1110700E0C71DB8F1010F7A
:1046F80033DBDDE902010022002300F0C1FB2CD2EC
:104708001C2102A800F0D4FBDDE9020100F058FCEE
:10471800A8F10708B8F1010F814609DB00F07CFC1D
:1047280002460B46DDE9020100F08EFCCDE90201EC
:10473800F81D072105E009F00F0200F8012D4FEAE6
:104748002919B9F1010F01DB491EF4D5491E5CBFD7
:10475800002200F8012DF9D5C7E70DF11100391A2B
:10476800B142B8BF0E4636B230000DF111072FD452
:10477800884206DA04A9411849780829A8BF0F21F8
:1047880000DA002104AA821800E0761E12F8013926
:10479800401E8B42F9D00F2904D104A941184A7848
:1047A800521C4A70002802D504AF761C2D1D36B263
:1047B800701E0DD4C1190A783032D2B23A2A03DBFE
:1047C8009DF838303A3B9A18401E01F80129F2D575
:1047D800206B002840F1ED80701E2063E9E0DDE9E0
:1047E80002010022002300F033FB3CBF81F00041AE
:1047F800CDE902012DB247F2975068434B49DFF8E3
:10480800309190FBF1F52DB2C5F1070ABAF1010F0D
:1048180090461CDBDDE902675FEACA7007D54246AD
:104828004B463046394600F0CFFC06460F46404618
:10483800494642464B464FEA6A0A00F0C5FCBAF1BF
:10484800000F80468946E7D1CDE9026724E0CAF126
:10485800000A0026374F14E05FEACA7007D54246BF
:104868004B463046394600F0AFFC06460F464046F8
:10487800494642464B4600F0A7FC4FEA6A0A804682
:104888008946BAF1000FE7D1DDE9020132463B461D
:1048980000F06CFDCDE90201BBF1660F216BDFF87A
:1048A80098900CBF05F10A0006204618142EA8BFE0
:1048B800132630208DF810000DF11107012E3DDB75
:1048C800DDE9020100F092FB07F1080104220A2346
:1048D800B0FBF3F303EB8307A0EB4700303001F89C
:1048E800010C0A20B3FBF0F000EB8007A3EB4703B1
:1048F8003033521E01F8023DE9D1083E012E01F184
:104908000807DBDBDDE9020100F070FB00F08EFB3D
:1049180002460B46DDE9020100F096FB00224B46F9
:1049280000F052FCCDE90201CAE700BFA0860100F1
:10493800000024400000F03F84D797410DF111009A
:10494800381A0DF1110702E0401E6D1E7F1C3978E0
:104958003029F9D0BBF1660F02D12DB2691C04E0F1
:10496800BBF1650F0CBF01210021226B8E1836B2F6
:10497800B042B8BF064636B231001AD4814204DAD2
:10498800C85D3528A8BF392000DA3020CA19521E60
:1049980000E0761E12F80139491E8342F9D0392801
:1049A80002D1C85D401CC855002902D57F1E761C5F
:1049B8006D1C2DB29DF83810009533B23A4620464A
:1049C80000F003F80FB0BDE8F08F2DE9F04305467D
:1049D8001E46D5F83080012E85B08946174602DA82
:1049E80001260FF2902749F02000BDF930406628D3
:1049F80008BF641C17D0672840F0828014F1040FA8
:104A0800C0F28480444580F2818095F83800641CA7
:104A1800000702D44645B8BFB04624B2B8EB040834
:104A280048BF4FF0000824B2E868A969012C25DACC
:104A38004A1C30230B54B8F1010F03DA95F83810EB
:104A4800090702D52E211154521C18EB040FB8BFC8
:104A5800C8F1000424B2A0446142B045AA61696269
:104A6800B8BF4646AB6936B2EE61324639461818C9
:104A7800FDF77CFBA8EB0600A862C1E00818A64277
:104A880018DA32463946FDF771FBA9697118A01B7F
:104A9800B8F1010FA961686203DA95F838000007D8
:104AA80005D5EA682E208854E869401CE861C5F8F5
:104AB8002880A5E022463946FDF758FBA86920184A
:104AC800361BB8F1010F03DA95F83810090703D53A
:104AD800EA682E218154401CA86136B2B045B8BF9F
:104AE8004646E868AB6936B23246E1191818FDF750
:104AF8003DFBA8693018A861A8EB060068627FE052
:104B0800B9F1610F16D14FF0700918E0464504DA83
:104B180095F83810090758BFB046B8F1010848BFE2
:104B28004FF00008B9F1670F14BF4FF045094FF077
:104B3800650904E0B9F1410F08BF4FF05009A969B0
:104B4800E86817F8013B0B544A1CB8F1010F05DA65
:104B580095F83810090758BFAA6117D52E211154A6
:104B6800531CB8F1010FAB6110DB761E36B2B045AD
:104B7800B8BF464636B2324639461818FDF7F6FA37
:104B8800A8693018A861A8EB06006862E868A969F6
:104B98000918200081F8009003D42B2048708F1C3E
:104BA80003E02D224A708F1C644200260DF108088C
:104BB80008E00A2200A800F004FD019808F8010B9B
:104BC800761C009C21B20129F3DA022E06DA49F09C
:104BD8002000652804BF302007F8010B4EB93020AB
:104BE80007F8010B07E0761E02A8305C303007F8A2
:104BF800010B012EF7DAE868A9690818381AE86184
:104C080095F8380000F0140010280DD16869A969DA
:104C18000818696A0818E9690818A96A0818696B00
:104C28008842BCBF081A286205B0BDE8F083F8B511
:104C380004460D4616461F46002004E0E86A401C5C
:104C4800E8627F1E002047B116F8011BA868A0473C
:104C58000028A860F2D14FF0FF30F2BD686A6C748A
:104C68007A4C00006E616E004E414E00696E66001F
:104C7800494E4600300000000278C9B28A421AB193
:104C88001CBF10F8012FF9E718BF0020704700007B
:104C980000F10103810704D010F8011B89B18107D5
:104CA800FAD10268B2F10131914311F0803F04BF9B
:104CB80050F8042FF6E710F8011B11B110F8011B8A
:104CC800FBE7C01A70470000C9B2830706D0521E1E
:104CD80022D310F8013B9942F7D11FE0083A13D3C9
:104CE80002F1040241EA012141EA014150F8043B82
:104CF800121F21BF4B40A3F1013C2CEA030C1CF00E
:104D0800803FF3D0C9B2001F083210F8013B521E91
:104D180028BF91EA030FF8D818BF0120401E70473A
:104D28001B4213D1094236D12AB18446B0FBF2F0B6
:104D380002FB10C2704700F04BBCFCD300220023DA
:104D480070470B000200002100207047904271EB71
:104D5800030CF6D370B5B1FA81F4B3FA83F52C1BC2
:104D6800A340C4F1200532FA05F63343A2405FF0B0
:104D78000046E64002E05B085FEA3202841A71EB03
:104D8800030524BF204629467641F4D302000B00D0
:104D98003000002170BD012ACFD970B5140C20D085
:104DA800B1FA81F4B2FA82F5C4F120046419B4F1BD
:104DB8002006D6D3B2405FF00044F440002502E05C
:104DC80052085FEA3303C61A71EB020E24BF30465D
:104DD800714664416D41F3D302000B0020002900A5
:104DE80070BD0C46B1FBF2F102FB11452D0445EAFA
:104DF8001045B5FBF2F402FB145580B240EA0545B4
:104E0800B5FBF2F002FB105240EA044070BD30B42A
:104E1800436803F0004201211B031B0B436004BFDE
:104E28000368002B08D10DE00368DD0F45EA440450
:104E380044605B000360491E4468E302F4D5230321
:104E48001B0B436043681A434260084630BC7047F6
:104E58004FF4001C1CEB410F94BF1CEB430F09E0FF
:104E680041EA030C50EA4C0C52EA0C0C03D299426A
:104E780008BF9042704714BF8B42824270470000BF
:104E88004FF4001C1CEB410F94BF1CEB430F09E0CF
:104E980041EA030C50EA4C0C52EA0C0C03D28B4248
:104EA80008BF8242704714BF994290427047000081
:104EB80070B504460D466068C0F30A5040F2FF71B1
:104EC800884207D16068000304BF2068002817D013
:104ED800022070BD20B92046FFF799FF012868DA43
:104EE800012D0FDB40F2FF71091A8D420AD3606869
:104EF800002847BF0020304900203049C4E900019C
:104F0800012070BD4142A942616806DA6FF31E5163
:104F1800401941EA0050606042E0401E636845194C
:104F2800012205F1350062F31F53352801F00041D5
:104F3800636003D361600020206070BD002215F11A
:104F48001F0F04DA22682360002020356060684261
:104F580014D0521E25689241C0F12003D2439D40CF
:104F680045EAD272256825FA00F6656805FA03F362
:104F780033432360636823FA00F56560606808437B
:104F8800B2F1004F606003D80DD12078C0070AD570
:104F98002068401C2060206828B96068401C606058
:104FA8004FF0FF3070BD6068884204BF2068002859
:104FB800F6D1002070BD00BF0000F0FF0000F07FB8
:104FC800F446400D40EAC120490006D200F014F82A
:104FD800004248BF6FF00040604700F00DF84FF006
:104FE800004188428CBF084640426047400D40EA75
:104FF800C120490080F00D8040F00040490DA1F526
:105008008061491C05D4D1F11F0154BFC840C017A5
:1050180070474FF000007047010040F10980F446E6
:10502800404200F005F851F000416047010000BF20
:1050380009D0B0FA80F18840C91CC1F5846109051E
:1050480001EBD02140057047F0B44FF0004591EADC
:10505800030F44BF6B4000F0BDBA00BF841A71EB68
:10506800030604D26E40001BB141121973414FF47C
:10507800001C1CEB410F34BF7CEB430684E00C0D95
:10508800A4EB1356362E7DDC012E43DC45EAC32300
:1050980043EA525312BFD20292025B08240545EA42
:1050A800C12141EA5051D2EBC020994125D407D102
:1050B800B0FA80F610FA06F164D00020203608E035
:1050C800B1FA81F6B140C6F1200220FA02F211438A
:1050D800B0404FEAF474B4EB465434F001064FEA9A
:1050E80074040AD8D6F50016760D04F00044F04092
:1050F80061FA06F25040F1404840C00A40EA415087
:1051080021F0004128BF5FEA500550F1000044EB50
:10511800D12137E045EAC323DB0A45EAC121C90AA0
:10512800B6F120050EDD42EA0242120CC5F1200656
:1051380003FA06F6EB4042EA06056D42984161F132
:1051480000010DE062FA06F5F240554063FA06FCEC
:1051580082EA0C02F3405A406D42904161EB030130
:1051680011F4801F05D1641E620502D06D00404114
:10517800494121F48011430875F1004350F10000C2
:1051880041EB0451F0BC70471CEB410F15D223F0E2
:10519800004352EA43060BD04FEA4C0CBCEB410FDC
:1051A80004D80C0D661E342EB7DDEBE7801A994142
:1051B80050EA410608BF0021E4E708BF1CEB430F93
:1051C80028BF6FF00001DDE7B0B581EA030C0CF0F1
:1051D800004C40F2FF7515EA11541DBF15EA13572C
:1051E800AC42AF4239E0E41923EA455343F4801353
:1051F800C90241F0004141EA505EC7021100A7FB15
:10520800020200284FF00000EEFB01204FF00001E1
:10521800E3FB072118BF42F0010240180021494171
:10522800E3FB0E01A4F580640F0302D25200404153
:10523800494154F101046CDD470872F1004250F114
:10524800000051EB0451A1F580115CBF41EA0C014B
:10525800B0BD4CEA05510020B0BD05EA1357AC4279
:1052680014BFAF4241E050EA410E1CBF52EA430E60
:1052780002E061460020B0BD24423C441BD15FEAF5
:10528800070EF6D0090302BF01460020AEF1140E46
:10529800B1FA81F7AEEB070401FA07FE0C37C7F144
:1052A800200100FA07F7C8404EEA000E23EA4553EA
:1052B80043F48013A2E733F00043B3FA83F704BF43
:1052C800B2FA82FE77440B3FE41BB7F1200E2FBFE2
:1052D80002FA0EF3BB40C7F1200E22FA0EFE38BFC9
:1052E80043EA0E03BA40641C82E750EA410E14BF39
:1052F80052EA430E6FF000014FF4001717EB430F0B
:105308008ABF194617EB410FB5E74CEA0551002053
:10531800B0BDD4F10104B4F120070FDAC4F12007BD
:10532800520828BF42F0010210FA07F501FA07F700
:10533800E1BF2A43E0403843E1400FE0352C98DCD8
:10534800C7F1200452EA400220FA07F218BF42F0DF
:10535800010231FA07F0A1400A43002172F100422C
:1053680050F1000051EB0C01B0BD00002DE9F041F7
:1053780040F2FF7581EA030C0CF0004C15EA115459
:105388001DBF15EA1357AC42AF42E9E0BC41C1F377
:105398001301C3F31303801A994143F4801304D211
:1053A800641E4000494180185941C90241EA5051E0
:1053B800B1FBF3F603FB1611A2FB0675D7EBC02071
:1053C800A94102D2761E80185941C90241EA5051BA
:1053D800B1FBF3FE03FB1E11A2FB0E75D7EBC02039
:1053E800A94103D2AEF1010E80185941890241EA60
:1053F8009051760546EA8E2EB1FBF3F603FB1611A3
:10540800A2FB0675D7EB8020A94102D2761E801830
:105418005941C90241EA50514EEA060EB1FBF3F672
:1054280003FB1611A2FB0675D7EBC020A94102D2D7
:10543800761E80185941C90241EA5051B1FBF3F771
:1054480003FB1711A2FB0735D3EBC020A94167F175
:1054580000070CBF004247F0010766F3D5274FEA63
:105468001E31B80814F5806414DDBD0775F10042DB
:1054780050EB0E5051EB045111F5801F5CBF41EA0F
:105488000C01BDE8F0814CF07F6141F0E041002063
:10549800BDE8F081BD076D0840EA0E5041F4801167
:1054A800D4F10104B4F120060ADAC4F1200602009E
:1054B800E04001FA06F3E1401843B24015430EE01C
:1054C800342C14DCC6F1200445EA40056D0820FAA6
:1054D80006F2154321FA06F0A1400D43002175F1AB
:1054E800004250F1000051EB0C01BDE8F0810020B2
:1054F8005FEA0C01BDE8F081CFB992185B41B3FABD
:1055080083F704BFB2FA82F6BF190B3FB7F1200642
:105518002FBF02FA06F3BB40C7F1200622FA06F6AF
:1055280038BF3343BA401CB1E419641E2FE77F42E9
:1055380031F00041B1FA81F404BFB0FA80F6A41941
:105548000B3CB4F120062FBF00FA06F1A140C4F1CC
:10555800200620FA06F638BF3143A0403C1B16E768
:10556800AC421ABF05EA1357AF4214E050EA4106AD
:105578001CBF52EA4306BFE750EA4107304661467E
:105588001CBF41EA0551BDE8F08152EA430C08BF4F
:10559800C143BDE8F08100204FF4001616EB410F1F
:1055A80098BF16EB430F08BF16EB410F24BFC1434A
:1055B80005E016EB430F0CBF61464CEA0551BDE808
:1055C800F08191FBF2F303FB1211C0E9003170473F
:1055D80070470000841A71EB030603D2001BB14127
:1055E800121973414FF4001C1CEB410F34BF7CEBC4
:1055F800430443E00C0DA4EB1356352E50DC45EA6A
:10560800C323DB0A45EAC121C912B6F120050DDD25
:1056180063FA05F6EB4086EA0305124218BF45F027
:105628000105C01851F100010CD213E062FA06F529
:10563800F2405540F3415A40B340F3405A40801875
:10564800594107D349085FEA30005FEA350528BFAA
:1056580045F0010501F58011420875F1004250F14D
:10566800000041EB0451F0BC4FF4001C1CEB410F4F
:1056780038BF70470020090D090570471CEB410F22
:1056880010D252EA43060BD0BCEB410F05D80C0DE3
:10569800AB43661E342EB5DD02E0AB43801859419A
:1056A800F0BC7047F0BC704780B5FBF74EFFFCF7C5
:1056B800D1FCFCF7DFFC8005800DDFF8741708606B
:1056C800DFF87007FCF76BFC012801D100200BE024
:1056D800DFF864070078002804D0DFF8601700209E
:1056E800FCF7F2F95FF0FF3002BD10B54FF47A71A4
:1056F800DFF84007FCF772FC012802D07FF00200B7
:1057080017E0DFF82C0700680400DFF824070068BA
:10571800401CDFF81C170860DFF8140700688005D4
:10572800800DDFF80C170860DFF80807FCF774FC39
:10573800200010BD002001000A2913DADFF8000755
:10574800182303FB01000200002010800020906055
:105758000020D060002010740020506100205060AC
:10576800491CE9E70020704710B50400FBF7EDFE7F
:10577800606110BD10B50400E068002802D0E06840
:10578800FBF727FE0020E060002020740020208026
:105798000020A0600020606100206060002010BD33
:1057A800F8B504000027002005000A2D15DADFF8F7
:1057B8009006182101FB0500060096F91000002844
:1057C80009D101203074B460002070603000FFF708
:1057D800CBFF370001E06D1CE7E73800F2BD2DE98B
:1057E800F04104000D005FF00008002006000A2EBA
:1057F80016DADFF84C06182101FB0600070097F9B6
:10580800100001280AD1B868284015EA0401884226
:1058180004D13800FFF7A8FFB84601E0761CE6E798
:105828004046BDE8F08170B5002004000A2C21DA5A
:10583800DFF80C06182101FB0400050095F910009B
:10584800012815D1FBF781FE06006869301A42F27B
:10585800117188420CD3DFF8E0054078002804D0A5
:10586800DFF8E0150120FCF72FF92800FFF782FF89
:10587800641CDBE770BD2DE9F84F04002768DFF8EA
:10588800C8153800FFF7ABFF0500002D31D1C7F36D
:105898008040002819D13800FFF782FF0500002D4D
:1058A80027D1DFF894054078002804D0DFF89C154C
:1058B8000120FCF709F9DFF89805C069401CDFF8FA
:1058C8009015C8615FF0FF3009E1DFF86C0540789A
:1058D800002804D0DFF87C150120FCF7F5F8DFF884
:1058E8007005806A401CDFF8681588627FF0010047
:1058F800F5E000200600B80C10F00100002802D0E6
:10590800012879D0DDE02079062814D2DFF82805AF
:105918004078002804D0DFF840150120FCF7D4F8BF
:10592800DFF82C05806A401CDFF8241588622800FF
:10593800FFF720FFD2E0E868002811D0DFF8F8046C
:105948004078002804D0DFF814150120FCF7BCF8D3
:10595800DFF8FC04806A401CDFF8F41488621CE05D
:105968004FF48070FBF7BCFCE860E868002814D1AD
:10597800DFF8C4040078002804D0DFF8E41400201D
:10598800FCF7A2F8DFF8C804806A401CDFF8C014EE
:1059980088622800FFF7EEFEA0E05FF0040814F12B
:1059A80008000090E86810F10A0942460099484644
:1059B800FCF7DCFBE868D0F80A00FBF7C0FDE968F3
:1059C800C1F80A005FF0020914F10C0AE86810F146
:1059D800080B4A4651465846FCF7C8FBE868008958
:1059E800FBF79AFDE9680881002028800620060058
:1059F800C7F38720401C6860C7F387206968491E81
:105A0800884214D0DFF830040078002804D0DFF88A
:105A180054140020FCF758F82800FFF7ABFEDFF815
:105A28003004806A401CDFF82814886256E06868F1
:105A3800401E6860E8680089298822795118F6B202
:105A4800891B884214DADFF8F0030078002804D0B4
:105A5800DFF814140020FCF737F8DFF8F403806A45
:105A6800401CDFF8EC1388622800FFF783FE35E05E
:105A78002079F6B2B0EB0608F6B2301910F1080931
:105A8800E8682988081810F10E0A42464946504627
:105A9800FCF76CFB288821790818F6B2801B28804F
:105AA8002888E9680989884218D10022DFF8A013FC
:105AB800E868FDF789FD0020E8602800FFF75AFE36
:105AC8000CE0DFF874034078002804D0DFF89C135A
:105AD8000120FBF7F9FF2800FFF74CFE0020BDE886
:105AE800F28F30B585B004004FF47A7200A9DFF860
:105AF80080030068FBF75AFD0500012D02D0FFF76F
:105B080092FEF1E700A8FFF7B6FEEDE738B504000E
:105B18000D002A002100D6480068FBF73CFD01284B
:105B280002D05FF0FF3000E0002032BD2DE9F54FD4
:105B380089B00C00FFF7D9FD0600002E0AD5BE4833
:105B48004078002803D0CB490120FBF7BDFF7FF048
:105B58000100E3E006208DF80100D4F80A00000DEA
:105B680010F01F00FBF769FD8DF800009DF800009C
:105B7800FF2806D1D4F80A00000D10F01F008DF898
:105B880000000027D4F80A00400810F0F850074336
:105B98009DF8000010F01F0057EAC047B005800DBF
:105BA800074320899DF801100818401E082190FB22
:105BB800F1F0C0B257EA80279DF80100D0F1080043
:105BC8008DF802009DF80200218980B2884202D334
:105BD800B4F808B001E09DF802B0D4F80A00FBF769
:105BE800A2FC02902089FBF791FCADF80400042088
:105BF800079002A806900DF10C08079A06994046EE
:105C0800FCF7B4FA5FF002080DF104090DF1100A6F
:105C1800424649465046FCF7A9FA5FFA8BFB14F155
:105C28000E00059003A89DF8011011EB000A5A46D2
:105C380005995046FCF79AFA5FFA8BFB5D469DF88A
:105C480001001BEB0002D2B203A9380000F06BF987
:105C580000280AD078484078002803D086490120D7
:105C6800FBF732FF7FF00A0058E02089ADB2854289
:105C780050D22089ADB2401B082802DB5FF0080B28
:105C880002E02089B0EB050B5FF00008D4F80A00A9
:105C9800400810F0F85050EA08089DF8000010F08D
:105CA8001F0058EAC048B005800D50EA080858F4AB
:105CB80080282089ADB2401B5FFA8BFBB0EB0B004C
:105CC800C01D082190FBF1F0C0B258EA80285FFAA5
:105CD8008BFB1BEB05055A46D2B2ADB228195FFA09
:105CE8008BFBB0EB0B0010F10E01404600F01BF9E6
:105CF8000028BAD050484078002803D05F490120D6
:105D0800FBF7E2FE52488069401C514988617FF0E8
:105D18000A0003E02000FBF75CFB00200BB0BDE8A5
:105D2800F08FF0B583B004000D00FFF703FD0028E5
:105D38000AD041480078002803D051490020FBF7D9
:105D4800C3FE5FF0FF3070E0FFF7AEFC00280AD01A
:105D580039480078002803D04A490020FBF7B4FEF0
:105D68005FF0FF3061E0E4B2002C03D15FF478000B
:105D7800070010E0E4B2012C02D1002007000AE07D
:105D88002D480078002803D03F490020FBF79CFEEF
:105D98007FF0010049E010214FF48070FBF7DBFB36
:105DA800334908603248006800280AD12248007840
:105DB800002803D035490020FBF786FE5FF0FF304E
:105DC80033E03348019006200090002340F2DC5273
:105DD80016A1304800F02AF90600002E0AD016480D
:105DE8000078002803D02C490020FBF76DFE5FF0F7
:105DF800FF301AE0FBF766FC2A003900C0B210F049
:105E08001F00C00400F04CF800280AD00A480078A7
:105E1800002803D021490020FBF756FE7FF00A0036
:105E280003E00B48FDF712FB0020FEBD43414E0086
:105E38002CDC002030DC002000000020C8A9000075
:105E480044D60020A4AF0000FF03F81F74AD000083
:105E58000800002098AD00009CB10000DCB30000F1
:105E6800C0A70000C4AF0000F0B30000BCAD000044
:105E780038DC0020F0A9000018AA000040AA0000A1
:105E880068AA0000A0A6000004B40000E4AF000067
:105E980034DC0020EB5A0000B8B1000004B0000068
:105EA800FEB504000D0016005D48056001205D493F
:105EB80008602020009020230022306840F4005120
:105EC80051F01001584800F0F6F80700FFB2002F13
:105ED80002D0FFB2380025E04FF48061524800F04C
:105EE8009EF90121504800F065F9002001905FF00B
:105EF800FF300090029840F47F4050F0FF0002907D
:105F0800029880B2029000A9474800F093F9070070
:105F1800FFB2002F02D0FFB2380003E0424800F081
:105F280063F90020FEBDF0B585B004000D00160031
:105F3800009810F0070050EAC4000090039850F44D
:105F480080100390F6B2039866F313400390002084
:105F58000700F6B2B74205DA785700A97918087130
:105F68007F1CF6E730480068C06810F1010F03D1C4
:105F78000120FCF73DFAF5E700A92B4800F056FA96
:105F88000100012901D1002000E0012005B0F0BD89
:105F980070B58AB000200090234800F046F904004C
:105FA800600504D54FF480611F4802681160E00461
:105FB8002FD500251C4800688068002824D001A936
:105FC800194800F0E3F90600F6B2012E1CD1019839
:105FD800C00805900498000C10F00F008DF8180008
:105FE8000020C0B2082809DA01A9C0B2411809790D
:105FF80005AAC0B282181172401CF2E76D1C00A9F4
:1060080005A8FFF783FDD5E74FF4805106480268DD
:1060180011600098002801D0FDF706FE0AB070BD97
:106028000CDC002030000C42F4DB00202DE9F043AA
:1060380085B004000D0016001F00DDF83080DDF883
:1060480034900020039000200290CDF80490CDF801
:1060580000803B00320092B229002000FCF7C2F811
:106068000100012902D05FF0FF3000E0002005B0F8
:10607800BDE8F083012110F01F029140DFF84422AF
:1060880040B2430942F823107047012110F01F0263
:106098009140DFF8342240B2430942F82310704798
:1060A800012110F01F029140DFF8202240B243097D
:1060B80042F8231070472DE9F04788B005000E001C
:1060C80017009846109CDFF80802006850F400504A
:1060D8007F4908601020FFF7D8FF1020FFF7E0FF86
:1060E8007B48006830F40050794908607948A84234
:1060F80001D001205BE07848286085F804806C7145
:10610800019810F0070001900020029000200390F1
:1061180000200490002005900020069000200790A1
:106128005FF080100090002082465FFA8AFABAF188
:10613800200F08D200AA5146C9B2664800F0D2F82A
:106148001AF1010AF1E7002E2BD13868C0F30320B9
:10615800022801D202202AE03868C0F34210002841
:1061680009D03868C0F34000002806D03868C0F36A
:106178004210012801D1032019E03868C0F38100DA
:1061880081463868C0F30320484504D33868C0F313
:106198004210484501D2042009E03868296888611E
:1061A80001E028688661002029684860002008B05E
:1061B800BDE8F087026852695208520003685A61C4
:1061C80049B210290CD1424A126852F40052404B8D
:1061D8001A603F4A126832F400523D4B1A6002E0DE
:1061E80049B202685161704710B504000020216867
:1061F80008602068406950F001002168486110205B
:10620800FFF738FF2068406850F4805021684860E4
:106218002068406850F001002168486010BD02689D
:1062280052680A4303685A607047006840688008EB
:106238008000704730B4020000231079002801D193
:1062480007203CE01079D0F120000400E4B2202CB3
:1062580033D21068E4B210EB44104D68C0F83452E1
:106268001068E4B210EB44100D68C0F830521068A2
:10627800E4B210EB44108D68ADB2C0F83852106823
:10628800E4B210EB44108D682D0CC0F83C52E4B217
:106298001F2C07D21068E4B210EB44100F4DC0F861
:1062A800205206E01068E4B210EB44100C4DC0F820
:1062B800205200200300641CC8E71800C0B230BC9C
:1062C8007047000000E100E080E100E080E200E0CB
:1062D80048800340F4DB002000500140E8008000C3
:1062E800A800800030B40300C9B21879D0F12000AA
:1062F800814201D3052047E05068C0081C68C9B234
:1063080014EB41141D68C9B215EB4115D5F8245298
:1063180015F0070555EAC000C4F824021868C9B288
:1063280010EB4110D468C0F82C421868C9B210EBC1
:1063380041109468C0F828421868C9B210EB41109F
:106348005469C0F834421868C9B210EB4110146996
:10635800C0F830421868C9B210EB41109469C0F80F
:1063680038421868C9B210EB4110D469C0F83C42F1
:106378001868C9B210EB4110146844F4000454F0D2
:10638800A804C0F82042002030BC704730B4020096
:1063980000231079002801D1072045E01079D0F1B9
:1063A80020000400E4B2202C3CD21068E4B210EBC8
:1063B8004410D0F82002C00732D51068E4B210EBC0
:1063C8004410D0F82402C0080D6815F0070555EAF6
:1063D800C00008601068E4B210EB4410D0F82C023A
:1063E80088601068E4B210EB4410D0F828024860C6
:1063F8001068E4B210EB4410D0F82002C8601068AE
:10640800E4B210EB44101568E4B215EB4415D5F866
:10641800205255F00105C0F820520120030001E088
:10642800641CBFE71800C0B230BC7047F8B5040060
:106438000D0000266079002801D107203AE0607934
:10644800D0F120000700FFB2202F31D220000068D1
:10645800C0680100F940C80728D42868C008216826
:10646800FFB211EB07112268FFB212EB0712526A52
:1064780012F0070252EAC00048622068FFB210EB2F
:106488000710A968C1622068FFB210EB071069689D
:1064980081622068FFB210EB0710E96841F400013F
:1064A80051F0010101620120060001E07F1CCAE7EA
:1064B8003000C0B2F2BD00680069C0F30720704721
:1064C800012110F01F029140DFF8E82540B243098E
:1064D80042F823107047012110F01F029140DFF8A5
:1064E800D82540B2430942F823107047012110F023
:1064F8001F029140DFF8C42540B2430942F8231037
:106508007047F8B5040094F90400FFF7E4FF842607
:1065180000273A0031002000FAF72EFE01206062C1
:1065280000200500ADB2082D07DA5FF0FF30ADB2EC
:1065380014EBC50148636D1CF4E7DFF88405844259
:1065480018D1DFF88005206002202071DFF8780577
:10655800006850F40070DFF8701508600220FFF73B
:10656800C5FFDFF86405006830F40070DFF85815DF
:10657800086017E0DFF85405206003202071DFF879
:106588004805006850F48060DFF83C150860032077
:10659800FFF7ACFFDFF83005006830F48060DFF803
:1065A80028150860206800684000400821680860D5
:1065B800F1BD2DE9F84F0400206800680500206847
:1065C800806906002068406807002068806A804665
:1065D8002068006B81462068406B82462068C0694D
:1065E8008346DFF8DC0484421ED1DFF8D80420603B
:1065F80002202071DFF8D004006850F40070DFF842
:10660800C81408600220FFF771FFDFF8BC040068B7
:1066180030F40070DFF8B0140860206800684000AB
:106628004008216808601DE0DFF8A004206003200E
:106638002071DFF89404006850F48060DFF8881453
:1066480008600320FFF752FFDFF87C04006830F48D
:106658008060DFF874140860206800684000400813
:10666800216808606D086D002068056020688661F3
:10667800206847602068006850F0010021680860C1
:106688002068C0F828802068C0F830902068C0F8DA
:1066980034A02068C0F81CB0BDE8F18F2DE9F041A6
:1066A80005000E0017009846069C95F90400FFF7B0
:1066B80012FF002085F88000286800684008400024
:1066C800296808602868006850F002002968086096
:1066D8002868006850F001002968086076B2082E22
:1066E80027DA002F08D0B7F1007F05D0B7F1807FF7
:1066F80002D0B7F1407F07D1DFF8D413394376B21F
:1067080015EBC602516306E0DFF8C813394376B2C9
:1067180015EBC602516376B215EBC60181F8384015
:106728005FEA5801491E080076B215EBC60181F8E8
:10673800390095F90400FFF7C3FEBDE8F08170B594
:1067480004000D0094F90400FFF7C5FE2068806876
:1067580010F004000600002E02D02000FFF729FFE9
:106768002068006840084000216808606DB214EB9A
:10677800C500406B216808606DB214EBC50090F845
:106788003900216888616DB214EBC50090F83800B3
:10679800216848602068006850F00100216808609E
:1067A8002068C0690121A94008432168C86194F99B
:1067B8000400FFF785FE70BD30B4046824686FF3E9
:1067C800172454F4807405682C600468E46A54F053
:1067D8000C040568EC62046861610468A46814F03C
:1067E80001042300002B05D10468A46814F00104F7
:1067F8002300F7E70468A46814F002042200002AC2
:1068080005D10468A46814F002042200F7E70068C0
:10681800006930BC7047002102689268D2050CD428
:106828000269C3689A4208D2826803699A5C03685D
:106838005A610269521C0261EEE70269C3689A4212
:1068480010D302689268D2050CD4C26983699A424F
:1068580008D24269C3699A5C03685A61C269521CCA
:10686800C261EEE7426A002A12D00269C3689A42FE
:106878000ED3C26983699A420AD302689268D20524
:1068880006D4202904D2002203685A61491CF4E77F
:10689800704710B582B0040094F9800002280DD129
:1068A80020688068400628D4206800690090606FDE
:1068B8000028F5D00098616F8847F1E794F98000C7
:1068C800012812D120688068400616D42068006923
:1068D8000090206BE16A884203D20098A16A226B7B
:1068E8005054206B401C2063ECE720688068400609
:1068F80003D4206800690090F7E713BD70B582B033
:106908000400206810F120052868800733D594F921
:10691800800002280DD120688068400628D42068AD
:1069280000690090606F0028F5D00098616F884773
:10693800F1E794F98000012812D1206880684006A8
:1069480016D4206800690090206BE16A884203D25F
:106958000098A16A226B5054206B401C2063ECE71E
:1069680020688068400603D4206800690090F7E733
:1069780002202168C8602868C0070DD594F98000F6
:10698800022803D1A06F2168486102E02000FFF7C8
:1069980042FF01202168C8602868C00617D520007A
:1069A800FFF777FF206A002806D0216BA06A226AC9
:1069B80090472000FFF72FFF012060622068806A5F
:1069C80030F010002168886210202168C8602868AB
:1069D80040070BD52068C06A50F004002168C862DF
:1069E8002000FFF7E6FD04202168C860286800073A
:1069F80021D52068C06A50F008002168C86294F95F
:106A0800800002280BD1206800686FF3172050F42B
:106A1800807021680860A06F2168486108E094F9D7
:106A28008000012804D1002020612000FFF7F3FE38
:106A380008202168C860286880062FD52000FFF745
:106A480028FF206B0600206A002810D00020606212
:106A5800002060610020A0610020E0611020216812
:106A6800C8602068806A50F01000216888620020A1
:106A780020612068C06A50F00C002168C8622000BC
:106A8800FFF7C9FE00202063E06F002803D0310023
:106A9800A06AE26F904720202168C86073BD80B566
:106AA8000748FFF72BFF01BD80B50B48FFF726FF0E
:106AB80001BD000000E100E080E100E080E200E0CC
:106AC80048D90020001000404880034000100140D1
:106AD8000201003402010030CCD90020012110F05D
:106AE8001F029140DFF80C2340B2430942F82310FB
:106AF800704710F0704203031B0B12EB4312C9B22C
:106B080012EB810212F1007201231360704710F03A
:106B1800704203031B0B12EB4312C9B212EB810242
:106B280012F1007200231360704710F070420003E6
:106B3800000B12EB4010C9B210EB810010F100708D
:106B48000068C0B2704770B504000D00160032002E
:106B5800D2B22900200000F0ACF8032120683030C0
:106B6800FFF7D5FF022120683430FFF7D0FF00215E
:106B780020683830FFF7CBFF0FF27930606270BDC4
:106B8800F0B40023DFF86863B04203D0DFF8D463C1
:106B9800B0421ED100291CD0002A1AD00668367DC2
:106BA8003500467B2E434673AE0610D51026102AB4
:106BB80000D2160000273C00B44207D25F5CD0F830
:106BC80000C08CF800705B1C641CF5E7121B002ADF
:106BD800E4D1F0BC704780B5DFF88C0300F00CF905
:106BE80001BD80B5DFF87C0300F006F901BD2DE991
:106BF800F04704000D00BE48844203D0DFF8640368
:106C0800844254D1A56000F0C5F9B948844204D142
:106C1800DFF858030068824603E0DFF85403006891
:106C280082465FEACA00B0FBF5F080465FEA58008A
:106C38000700B8090600402000FB1670814618EBD3
:106C48000900802101FB1600B0EB4909B6F5803F29
:106C58002DD2022E17D3072120680C30FFF749FFE9
:106C6800300A2168087120680670072120680C30F6
:106C7800FFF74DFF072120683030FFF73AFF206803
:106C880080F83C9013E0072120680C30FFF731FFB3
:106C9800300A2168087120680670072120680C30C6
:106CA800FFF735FF072120683030FFF730FFBDE8D8
:106CB800F08770B504000D0016008D48844214D189
:106CC8005FF0804020600A202071AA48006850F0D8
:106CD8008000A84908600A20FFF700FFA54800685F
:106CE80030F08000A349086012E0A34820600B2020
:106CF8002071A048006850F480709E4908600B20FD
:106D0800FFF7ECFE9B48006830F4807099490860F2
:106D1800002021680871002021680872012120687C
:106D28000830FFF7E6FE022120680830FFF7E1FE91
:106D3800002120680830FFF7DCFE042120681030AD
:106D4800FFF7E5FE052120681030FFF7E0FE01217E
:106D580020683430FFF7DBFE002120683430FFF76D
:106D6800D6FE012120683830FFF7D1FE05212068C2
:106D78003030FFF7CCFE062120683030FFF7C7FE21
:106D8800072120683030FFF7C2FE03212068383021
:106D9800FFF7BDFE0020216881F84400002021682B
:106DA80081F848000020216881F84C002900200063
:106DB800FFF71DFF20680673A56026730020606139
:106DC800002020610020A061002020620020606275
:106DD8000020E0610020A0620020E0620020206323
:106DE800002060630020A0630020E063002060733F
:106DF80070BD000080E200E038B504003C488442E1
:106E080002D05848844271D12068007A10F00F00EF
:106E18000500EDB2280000280AD002280FD0032868
:106E280022D0042812D0062817D00C280ED05DE0F6
:106E3800A06A002802D02000A16A884756E0606A4C
:106E4800002802D02000616A88474FE0206A0028A5
:106E580002D02000216A884748E0E069002802D073
:106E68002000E169884741E0002120682830FFF7C9
:106E78005CFE002805D0E06A002802D02000E16A04
:106E88008847012120682830FFF74FFE002805D0E9
:106E9800206B002802D02000216B8847022120683F
:106EA8002830FFF742FE002805D0606B002802D08A
:106EB8002000616B8847032120682830FFF735FEE2
:106EC800002805D0A06B002802D02000A16B8847BD
:106ED800042120682830FFF728FE002805D0E06B41
:106EE800002802D02000E16B8847FFE731BD000091
:106EF80050DA002070B504001B48844202D01948BB
:106F080084422DD1206900282AD06069002827D022
:106F18002068007D0500607B28436073A80614D5AF
:106F280010216269A369D21A102A00D21100002325
:106F38001800884209D22369A669F35C2668337071
:106F4800A3695B1CA361401CF3E7A06961698842DF
:106F580006D10020606101212068001DFFF7D7FDE0
:106F680070BD000090DA002050DA002024010020D3
:106F780028010020488003400000014080B500F04F
:106F880095F85648006850F400705449086000F0BD
:106F980044FA01BD2DE9FC415148006810F08060B9
:106FA8000400002C48D14E48006810F480500600B8
:106FB800002E15D14B484C4908604A484B49086097
:106FC80048484B49086047484A49086045484A4983
:106FD800086044484949086042484949086031E026
:106FE80000A848490CC90CC0083908384648006848
:106FF800C0F38210070000A8385C80465FFA88F862
:10700800B8F1000F04D0B8F1020F0DD007D30FE08C
:1070180000F01AF80500280000F023F812E04FF4F9
:10702800004000F01EF80DE0384800F01AF809E0BA
:10703800364800F016F805E000F006F805002800CC
:1070480000F00FF8BDE8F381314A126812F004022B
:107058001100002902D12F4A100001E02E4A100029
:1070680070472149086021490860214908601D4985
:10707800204A1160204908602049086020490860BA
:107088007047264A126811000A004FF602039A4216
:1070980003D0234B9A4203D005E00122100004E0FC
:1070A8000222100001E000221000704710B5FFF71F
:1070B800E8FF0400012C02D100F002F8FFE710BD40
:1070C8000748006850F48070054908600448006863
:1070D80030F08060024908607047000014ED00E05D
:1070E800988003400024F40020010020240100209F
:1070F800280100202C01002030010020340100204C
:1071080038010020A0B500009C80034040420F00D9
:107118005081034040787D0180F0FA024C810340A1
:1071280002F80100012110F01F029140DFF86823E6
:1071380040B2430942F823107047DFF86003006843
:10714800704710B5DFF85803006880088000DFF842
:10715800501308600320DFF84C1308600020FFF785
:10716800E1FFDFF8440300680400DFF8400300682B
:10717800844204D2DFF83803DFF83813086010BD02
:10718800DFF82C03DFF82C130860704780B54FF444
:1071980082710A20FAF724F80120FAF797FADFF843
:1071A80018130120FEF7BDFD00F0B4F9DFF80C0359
:1071B80000900023DFF80823DFF80813DFF808033E
:1071C80000F03BFBFF23DFF8042305210020FAF73A
:1071D80041FAFF23DFF8F42205210220FAF73AFAF0
:1071E800FF23DFF8E42205210920FAF733FAFF2309
:1071F800DFF8D82205211F20FAF72CFA0220FAF727
:10720800B3FC0420FAF7B0FC0520FAF7ADFC052121
:107218004FF4007000F001FD01BD2DE9F04788B082
:10722800814604A8102100F035FD00270024002520
:10723800002003900026FBF7BCF903904FF4807000
:10724800FAF775FA804620214046FCF745F9A04830
:10725800FCF7FEFAFFF794FF9E480078002802D05A
:1072680000209C49087000200700FFB2082F10DAA0
:10727800FFB2380080B200F03DFD80B2000904A9D9
:10728800FFB221F81700FFF758FF4002FBD47F1C1C
:10729800EBE79148FFF70FF99049C880BDF81A004D
:1072A800FDF7C4FE00228E4BFDF78EFF00228D4BAA
:1072B800FEF75CF800225FF08043FDF785FFFDF7DD
:1072C8007FFE86498881BDF81000FDF7AFFE0022D9
:1072D800834BFDF779FF0022824BFEF747F8002227
:1072E8005FF08043FDF770FFFDF76AFE7B49488138
:1072F800BDF8140000F04CFD78490872BDF818007C
:1073080000F046FD754948720020744988730020D2
:1073180072498880122000F05DFF7049C87302200E
:10732800F9F7DEFF82460220AAF808000A208AF848
:107338000E0000208AF80F0064200290CDF804A007
:107348000020009068480368DBB267480268D2B240
:107358001F210220FAF7ECFA002802D05046FAF76B
:1073680038F80A20FBF744F85C48C17B5F48FCF713
:107378006FFAFCF733FB01005D48FCF769FAFCF78C
:1073880030FB01005B48FCF763FA092000F060FF5E
:10739800FBF70FF90500281B0600C82E15D32C0093
:1073A8004E48807C00280CD04C48807C401E4B49BD
:1073B80088744A48008A642807DA642047490882A2
:1073C80003E042F21070454908824448008AC82107
:1073D80048434FF47A71B0FBF1F103A8FAF7AEFF16
:1073E80035E770B504004FF48070FAF7A0F905008E
:1073F80020212800FCF770F84FF47A712800FAF77A
:1074080084FA0600002EF7D0300000F047FF01286C
:10741800F2D13000F9F7DDFFEEE780B5FFF791FE16
:1074280001BD00B583B001F0E9F8FFF7AFFE002019
:1074380001900420009000234FF480722E492F48B9
:10744800FEF7F4FD002001900320009000234FF484
:1074580080722B492B48FEF7E9FD0020019001209E
:10746800009000234FF4807227492848FEF7DEFD7C
:10747800002001900220009000234FF4807205A1A3
:107488002348FEF7D3FD42F2107014490882FAF738
:10749800E5FF07BD444D000080E200E08430014074
:1074A800145000401C50004000500040085000405C
:1074B80042DE15AC0C5000408C00002080B5000066
:1074C8003F7500002CDB0020D0DA002008000020E7
:1074D80054B50000DEDC0020F4DB002064DB002073
:1074E80000409F4000FEAF40D8B50000E8B400005F
:1074F80090B40000A4B4000088B500001B9C0000F4
:1075080090B50000AB99000098B500002372000008
:10751800EB73000080B501214FF40050FAF71BF817
:107528002649086025480068002802D15FF0FF302E
:1075380000E0002002BD01B54FF4C87200A91F4841
:107548000068FAF717F801BD70B582B004000D00A5
:10755800002C14D00026AE4211DA002200A91748E8
:107568000068FAF723F8012803D0C0212170641CB1
:1075780003E09DF800102170641C761CEBE773BDD6
:1075880010B504000D480068FAF72BF8010000292F
:1075980002D15FF0FF3004E0A14201DA002000E0F0
:1075A800012010BD80B50123642200A903480068AA
:1075B800FBF774FD0128F6D101BD0000C8DC0020EE
:1075C8002DE9F04104000D001600002C02D060687F
:1075D800002802D17FF00A004EE000212800FCF7C5
:1075E80073F8D5F80A00F9F79EFFC5F80A0028894C
:1075F800001D28814FF47A71A248FAF7EFFC6768FA
:107608007FF03F00396888470020396888475FF075
:1076180000082889804524D218EB0500807AC02804
:1076280008D1DC2018EB050188727FF02400396846
:1076380088470CE018EB0500807ADB2807D1DD20AD
:1076480018EB050188727FF024003968884718EB29
:10765800050090F90A0040B23968884718F1010816
:10766800D7E77FF03F00396888472800F9F7B1FE6F
:107678008448FAF7D1FC0020BDE8F0812DE9F843F1
:107688000400884617001D0066683800471E002859
:1076980000F0D18098F8009018F10108A089B1682D
:1076A80088420ED278484078002803D077490120D4
:1076B800FAF70AFAE069401CE06100203073002004
:1076C800B06096F90C00002807D0022800F08E80E0
:1076D8002CD3032800F0A780D7E75FFA89F9B9F11E
:1076E800C00F08D07068002804D02900484640B26E
:1076F80072689047C9E7B06900280AD1002D04D103
:10770800A089F9F7EDFDB06103E0A089F9F7C0FDA4
:10771800B061B069002802D103203073B5E70020BA
:10772800B0600120307301203061AEE75FFA89F95B
:10773800B9F1DB0F02D102203073A6E75FFA89F9AD
:10774800B9F1C00F44D1B068002840D0B06808280B
:107758000ED24D484078002804D0B2684C49012028
:10776800FAF7B2F9E069401CE061002030738CE759
:10777800A06A401CA062B068001FB1690881B069A6
:10778800D0F80A00F9F7DBFEB169C1F80A00002158
:10779800B069FBF7C9FF00280FD03B4840780028A4
:1077A80005D0B06902893B490120FAF78DF9E069F3
:1077B800401CE0610020307367E72A002100B069AF
:1077C800FBF702FF0020B061002030735DE75CE743
:1077D8003069002802D00020306156E7B068411CAB
:1077E800B160B169401880F80A904EE75FFA89F9EC
:1077F800B9F1DD0F07D1B068411CB1607FF02401F9
:10780800B269801881725FFA89F9B9F1DC0F07D182
:10781800B068411CB1607FF03F01B2698018817285
:107828000120307331E75FFA89F9B9F1C00F01D14E
:107838000020307329E7BDE8F1832DE9F041040009
:107848000D0016001F00DDF8188013480068002896
:1078580005D10C48FAF7A3FB01200F4908606560C1
:107868006F602E600020A861002028734FF480709C
:10787800A0810A48A060C4F800802000FBF7E6FD5C
:10788800BDE8F08140DC00200000002018B40000B2
:10789800E0AD000090AA00003CDC0020C9750000A3
:1078A80038B504000D00A87A40070FD5DFF8A80303
:1078B8000078002804D0DFF8A4130020FAF704F9B0
:1078C800606A401C60627FF0040013E0A87A000739
:1078D8000FD5DFF884030078002804D0DFF8801380
:1078E8000020FAF7F1F8606A401C60627FF004003B
:1078F80000E0002032BD70B504000D001600B07A1B
:10790800C0071FD53089042808DAD3480078002832
:1079180004D03289D3490020FAF7D6F80021300084
:10792800FBF702FF002817D0CB480078002803D0C7
:10793800CD490020FAF7C8F8E869401CE8617FF0F3
:1079480065001DE0600607D5C3484078002803D0CD
:10795800C6490120FAF7B8F8B07A80070FD4E007D3
:107968000DD5BD484078002803D0C1490120FAF759
:10797800ABF8E869401CE8617FF0010000E00020F6
:1079880070BDF0B58BB00400FAF716F907A8FBF73D
:107998000CFE002802D05FF0FF3036E10898069010
:1079A80007A8C046C04610F1010F02D15FF0FF30B2
:1079B8002BE1A9480079002828D00798006805908D
:1079C8000698008904900698807AC0B203900698B9
:1079D800D0F80A00800F02900698D0F80A00C0F389
:1079E800052001900698D0F80A00C0F38530009071
:1079F8000698D0F80A00C0F304530698D0F80A0095
:107A0800C0F344629B490420FAF75EF8F9F75AFE7E
:107A18000699D1F80A10C1F30451C9B2C0B2814223
:107A28003BD00698D0F80A00C0F304501F2834D081
:107A38000698D0F80A00000D10F01F00F9F7F0FDC5
:107A48000700002F06D00798874208D10798807B47
:107A5800002804D10698F9F7BCFC0020D5E00020E6
:107A680006994118897A0AAA8154401C0428F7D338
:107A780000233A0006990A98F9F7A0FE00280AD0D0
:107A880075484078002803D07B490120FAF71CF894
:107A98000698F9F79EFC0020B7E006990798FFF7CB
:107AA800FFFE002804D00698F9F793FC0020ACE00C
:107AB8000698D0F80A00C0F38530FBF7E5FC06000D
:107AC800002E24D0F069C00521D5069A0799F069DF
:107AD800FFF711FF002804D50698F9F77AFC002073
:107AE80093E0002206A97069F9F744FD01280CD03B
:107AF80059480078002803D060490020F9F7E4FFCE
:107B08000698F9F766FC00207FE000207DE05C49DC
:107B18000698D0F80A00FAF729F90500002D59D17E
:107B2800002E04D10698F9F754FC00206DE0069A5F
:107B38000799F069FFF7DFFE002804D50698F9F7E2
:107B480048FC002061E00698D0F80A00800F800702
:107B58000700F9F7B7FDC0B260F35D670698D0F883
:107B68000A00C0F3446060F318570698D0F80A007A
:107B7800C0F3052060F393370698D0F80A00C0F3E5
:107B8800853060F30D270698807AC0B260F3070746
:107B9800002006994118897A09AA8154401C0428B2
:107BA800F7D339000998FAF76FF90500002D0CD1C1
:107BB80029480078002803D032490020F9F784FFCB
:107BC8000698F9F706FC00201FE070696861F06903
:107BD800E8610BE0069A0799E869FFF78CFE002830
:107BE80004D50698F9F7F5FB00200EE00698807A90
:107BF800800705D506992800F8F7F4FE002004E070
:107C08000699280000F012FD00200BB0F0BD10B559
:107C180004006420FFF7B5FEFBE77CB504000D0007
:107C28001948019000950023220092B209A1174833
:107C3800FEF7FCF90600002E0AD007480078002855
:107C480003D013490020F9F73FFF5FF0FF3000E051
:107C5800002076BD525445000000002074A00000AA
:107C6800DCA10000E4B000004CA9000090A70000CF
:107C780094A50000F4A3000070B300007CB20000DB
:107C880000FFFF3F04B100004CDC0020177C00001F
:107C980098B20000002200F001BD00000100481E5B
:107CA800002901D000BFF9E7704738B5040036480D
:107CB800006830F4807034490860102000908023F8
:107CC800002200213148FEF7E9FC00212F48FEF789
:107CD80036FDA4B221002D48FEF76EFD05002A48A6
:107CE800006850F48070284908602D052D0D280083
:107CF80080B232BD38B504000025A4B2082C1DDAC4
:107D08002148006830F480701F49086010200090F6
:107D18008023002200211D48FEF7C0FC00211B48DB
:107D2800FEF70DFDA4B221031848FEF745FD050036
:107D38001548006850F4807013490860280080B224
:107D480032BD80B51048006850F480700E49086054
:107D58004FF42C40FFF7A9FF6420FFF79FFF4FF473
:107D68001040FFF7A2FFB0F5406F0AD06420FFF77C
:107D780095FF4FF42C40FFF798FF6420FFF78EFF24
:107D8800EDE701BD000000008830014048D900201F
:107D980010B401000A4889B24A111056084A89B23B
:107DA80012EB61125278121A11F01F0352B2DBB2B1
:107DB80003FB02F46411201840B210BC70470000A5
:107DC80098000020BFF34F8FDFF85C04006810F4C0
:107DD800E060DFF858140843DFF84C140860BFF37C
:107DE8004F8F00BFFDE7DFF84814096851F4001110
:107DF800DFF83C2411604CF250310800002801D013
:107E0800401EFBE7DFF82814096831F40011DFF899
:107E1800202411604CF250310800002801D0401E87
:107E2800FBE7DFF80C14096851F48011DFF800242F
:107E38001160DFF8FC13096851F40021DFF8F02322
:107E480011604CF250310800002801D0401EFBE7B9
:107E5800DFF8DC13096831F40021DFF8D42311605E
:107E68004CF250310800002801D0401EFBE7DFF833
:107E7800C013096851F48021DFF8B42311607047FA
:107E88002DE9F04182B004000D00160000274CF2E5
:107E980050381FFA88F8B8F1000F4BD0DFF890037C
:107EA80000680121A1408843DFF884130860082096
:107EB800009040235FF000720021DFF87803FEF79E
:107EC800EDFB0021DFF86C03FEF739FC4421DFF8F5
:107ED8006403FEF771FC0021DFF85803FEF76CFC21
:107EE8000700FFB2FF2F19D1EDB2002D0CD02800EA
:107EF800451EC0B2002807D00021DFF83803FEF77E
:107F08005BFC3070761CF2E7DFF82403006801217F
:107F1800A1400843DFF8181308600BE0DFF81003EE
:107F280000680121A1400843DFF804130860B8F194
:107F38000108AEE71FFA88F8B8F1000F01D1FFF782
:107F480041FFFFB2FF2F03D10120DFF8EC120870C8
:107F58003800C0B2BDE8F68170B582B004000D00EB
:107F6800160000220021200040B2FFF789FFDFF849
:107F7800C00200680121A1408843AD49086008207B
:107F8800009040235FF000720021AA48FEF786FBAC
:107F98000021A848FEF7D3FB2800451EC0B20028E0
:107FA80005D03178A348FEF707FC761CF4E7A04813
:107FB80000680121A14008439D49086073BDF8B5D8
:107FC80004000F003878002825D0387806007F1C78
:107FD800F6B2112E01D304201EE000200500EDB2F8
:107FE800F6B2B54206D238789449EDB268547F1C8F
:107FF8006D1CF4E7914A3100C9B2200040B2FFF786
:10800800ABFF00220021200040B2FFF739FFFF2814
:10801800D8D0022000E00020F2BD00B5ADF21C7DF2
:10802800FFF7E1FE142000F0E9F8122000F0E6F86E
:10803800FFA8103082494FF44472FAF7A7F8FFA955
:1080480010311420FFF7BBFF002300220021142069
:1080580000F0A5F800A87B4940F20C42FAF796F820
:1080680000A91220FFF7ABFF0023002200211220F5
:1080780000F095F80DF21C7D00BD2DE9F0470700D2
:10808800884691469A46089C099D0A9E32206B496B
:1080980008706A4880F80180684880F802901FFAE2
:1080A8008AFA5FEA1A206549C870644880F804A013
:1080B80062484471614885716048C6715F4A082109
:1080C800380040B2FFF748FFBDE8F0873EB504002E
:1080D8000D00002300220021200040B200F05FF8CC
:1080E8000820029008200190002000900023002220
:1080F8002900C9B2200040B2FFF7BFFF37BDF8B56D
:1081080004000D0016001F0031204C4908704B4830
:1081180045704A488670BFB2380A4849C87047480F
:108128000771002045494871002044498871434A35
:108138000721200040B2FFF70FFFF1BD38B504005A
:108148000D00002300220021200040B200F027F893
:10815800002300222900C9B2200040B2FFF7CFFF58
:1081680031BD38B504000D0031203449087033485A
:10817800457001203149887000203049C8700020BE
:108188002E49087100202D49487100202B4988711B
:108198002A4A0721200040B2FFF7DEFE31BDF8B5BC
:1081A80004000D0016001F002020244908702348F1
:1081B8004570224886702148C770204A0421200053
:1081C80040B2FFF7C9FE1D4A0821200040B2FFF760
:1081D80057FEF1BD10B5040022201B4908701A4A49
:1081E8000121200040B2FFF7B7FE174A08212000FE
:1081F80040B2FFF745FE1448807810BD10B5040062
:10820800012012490870114A0121200040B2FFF7ED
:10821800A3FE0E4A0821200040B2FFF731FE0020DD
:108228000A49087010BD00000CED00E00400FA05D2
:108238008830014048D90020E1DC0020DCDB002048
:10824800489500003C8D000004DC0020FCDB002089
:108258003EB5040074480068744909680818F9F7BD
:108268003FF8050015F10E0000F0D6FA6E480068D8
:108278006E490968081828814FF47A7002900195B0
:10828800002000906A480368DBB269480268D2B2ED
:108298002100C9B20220F9F74BFB37BDF8B504003D
:1082A800002C02D15FF0FF30BCE0D4F80A00C0F324
:1082B80085305F490968884212D1208900280DD18C
:1082C800D4F80A00400E10F01F052800C0B2FFF7CE
:1082D800BFFF2000F9F77DF80020A3E00120A1E00E
:1082E800D4F80A00C0F3853052490968884201D0A1
:1082F800012097E02089002805D12000F9F769F8C6
:108308005FF0FF308EE014F10E0528780A3806D0A9
:10831800401E022819D9C01E012849D97EE0E67BF3
:108328002000F9F756F82089022802DA5FF0FF30BA
:1083380078E0F6B2002E03D01F20FFF789FF02E095
:108348000920FFF785FF00206CE02089042805DA62
:108358002000F9F73EF85FF0FF3063E0E878F8F7BF
:10836800BFFF0600002E05D12000F9F732F85FF0B4
:10837800FF3057E02878B073E878401C30813389A3
:1083880016F10F02B5F8011028780B38C0B200F0CA
:108398009FF90700002F06D44FF47A7300223100AA
:1083A8002000F9F76DFB2000F9F713F8002039E0F9
:1083B8002089042805DA2000F9F70BF85FF0FF3070
:1083C80030E00220F8F78CFF0600002E05D12000CF
:1083D800F8F7FFFF5FF0FF3024E02878B073012042
:1083E8003081EB789BB22A1DB5F8011028780D383A
:1083F800C0B200F0BDF90700002F03D5FF20F073CD
:10840800022030814FF47A73002231002000F9F7FE
:1084180037FB2000F8F7DDFF002003E02000F8F725
:10842800D8FF0020F2BD0000BCB50000C0B50000B8
:10843800C8B50000C4B5000010B440B2002808D583
:108448000A01664B40B210F00F04E31803F8042C3D
:1084580003E00A01624B40B2C25410BC704780B5B9
:1084680000F014FA0521012000F038FA5D48006890
:1084780050F002005B4908605A48006830F002007A
:10848800584908605748006850F00200554908608C
:108498000521132000F022FA0521152000F01EFA0C
:1084A8000521142000F01AFA0521122000F016FA0E
:1084B8000521082000F012FA0521192000F00EFA13
:1084C8000521092000F00AFA05210A2000F006FA21
:1084D80005211D2000F002FA02211A2000F0FEF901
:1084E80005210D2000F0FAF905210C2000F0F6F91D
:1084F80005210F2000F0F2F90521162000F0EEF911
:108508000521102000F0EAF90521112000F0E6F914
:108518000521002000F0E2F93248006850F480108C
:10852800304908602F48006850F480202D490860C1
:108538002C48006850F480502A490860294800688F
:1085480050F48000274908602648006830F400305D
:10855800244908602348006850F4803021490860A5
:1085680020480068400840001E4908601D4800680F
:1085780050F400501B4908601A48006830F4004065
:10858800184908601748006850F480701549086059
:108598001448006850F000501249086011480068FB
:1085A80050F000700F4908600E48006850F40070E1
:1085B8000C49086001BD80B50B48FDF7A2FF0820F3
:1085C800009040235FF0007200210748FEF766F82C
:1085D80000210548FEF7B3F801BD000018ED00E0E2
:1085E80000E400E08830014048D9002080B5FFF75A
:1085F80014FD00211220FFF769FD01BD80B50B2194
:108608001020FFF719FFFFF72AFFFFF7D4FFFFF746
:1086180098FBFFF7EBFF01BD13005A1E002B04D097
:1086280003680B60001D091DF6E7704711B581B09E
:108638000C0021000198F9F7DFFA00280BD514483F
:108648000078002803D013490020F9F73DFA2000EC
:10865800F8F7BFFE1AE001984069002816D00022FA
:1086680001A901984069F8F785FF01280BD008484F
:108678004078002803D008490120F9F725FA019825
:10868800F9F715FC02E000200199486113BD00BF0D
:108698000000002024B1000048AC000000B500BF75
:1086A800130096469446103928BFA0E80C50FAD813
:1086B8005FEA417C28BF0CC048BF40F8042BC907BB
:1086C80028BF20F8022B48BF00F8012B00BD00008E
:1086D8002DE9F04104000D0016001F00E4B2002C43
:1086E80003D0022C2BD015D33EE0ADB2BFB278191F
:1086F800042802D3D5F104000700BFB25348ADB235
:1087080015EB00083A0041463000F9F72FFD380014
:1087180080B22BE0ADB2BFB27819132802D3D5F1DD
:1087280013000700BFB24A48ADB215EB00083A0083
:1087380041463000F9F71AFD380080B216E0ADB2B4
:10874800BFB27819022802D3D5F102000700BFB2E0
:108758004048ADB215EB00083A0041463000F9F741
:1087680005FD380080B201E05FF0FF30BDE8F08120
:108778002DE9F04104000D0016001F00E4B22000AE
:10878800012802D0022820D042E0ADB2BFB2781949
:10879800132802D3D5F113000700BFB22C48ADB29D
:1087A80015EB00083A0031004046F9F7DFFCBFB28C
:1087B8003900280080B202000120002802D55FF0AD
:1087C800FF3027E0BFB2380024E0ADB2BFB278195D
:1087D800022802D3D5F102000700BFB21D48ADB28E
:1087E80015EB00083A0031004046F9F7BFFC0120BC
:1087F80019490870BFB23900280080B20200012070
:10880800002802D55FF0FF3004E0BFB2380001E075
:108818007FF00100BDE8F0812DE9F84304000F481E
:1088280005680B4E2A0031002000F9F79FFC0C4820
:108838000768DFF820800948006810EB04093A004F
:1088480041464846F9F792FCBDE8F183CCB50000F3
:1088580064DB002000FC0108D9DC0020B4B500006E
:10886800B8B50000012110F01F029140204A40B223
:10887800430942F823107047012110F01F0291406C
:108888001C4A40B2430942F82310704710B51A48F1
:10889800006850F48010184908601748006850F0C4
:1088A800F0701549086000200400202C09D21348F4
:1088B8002056FFF7D7FF11482056FFF7DDFF641C4D
:1088C800F3E70D48006830F0F0700B4908600A487B
:1088D800006830F480100849086010BD40B20200FA
:1088E800202A03D2064B53F8223019607047000043
:1088F80080E100E080E200E04880034044B10000ED
:10890800CC9E000070B5DFF8240400680600DFF88C
:10891800E0030068064016F002000500EDB2002DE5
:1089280001D000F0CCF816F001000400E4B2002CED
:1089380001D000F001F870BD10B5DFF8E40300784D
:10894800012804D002283AD005286AD0AAE0DFF826
:10895800B403008800282FD0DFF8A8030188DFF8C7
:10896800A003006800F097F90400DFF89803008876
:1089780084420ED2DFF88C030088001BDFF88413D2
:108988000880DFF87C0300682018DFF8741308609B
:1089980014E00020DFF86C130880DFF8700300682B
:1089A800002804D00220DFF87813087006E00320BE
:1089B800DFF86C13087001E000F056F97EE0DFF88C
:1089C8004C030068002829D0DFF840030168DFF86D
:1089D8003803006800F05FF90400DFF8300300682E
:1089E80084420ED2DFF824030068001BDFF81C1352
:1089F8000860DFF8140300682018DFF80C1308601B
:108A08000EE0DFF8EC02006840084000DFF8E012F2
:108A180008600320DFF80813087001E000F024F96B
:108A28004CE0DFF8E802006800281BD1DFF8F80204
:108A38000068002814D0B448DFF8EC1209688847A9
:108A4800B2490860B148006800280BD1A8480068FE
:108A580040084000A64908600320B149087001E0B9
:108A680000F002F9A9480068002809D1A048006868
:108A7800400840009E4908600320A949087010E09A
:108A8800A2480168A048006800F005F904009F4862
:108A98000068001B9D4908609B48006820189A4997
:108AA80008600BE092480068400840009049086060
:108AB800002000F0C5F800209949087010BDF8B5ED
:108AC8009B480068040014F40040050020000600DC
:108AD8009348007800280BD0022800F0A180C0F04D
:108AE8009F80042846D026D3052800F08680A0E081
:108AF800ADB2002D1ED0F6B2F12E05D037003800E9
:108B0800C0B200F0E8F815E00020834908808048EA
:108B18000068814909880E547F480088401C7E49B6
:108B2800088000207A4909687B4A1288505404203A
:108B38007B49087083E0ADB2002D1AD037006F482A
:108B48000078FFB2874210D100207349088070482E
:108B58000068714909880F546F480088401C6E49A5
:108B6800088004206E49087003E03800C0B200F0A5
:108B7800B2F864E0ADB2002D05D037003800C0B2BD
:108B880000F0A9F838E062480068634909880818C5
:108B980010F8010CF12811D15D4800685E49098878
:108BA8000E545B4800685C490988081810F8010CE5
:108BB80000F091F800205A4908701DE056480088D6
:108BC8005449098888420AD2300051490968524AF2
:108BD8001288505450490988491C4F4A11804E4800
:108BE80000884C490988884206D14B48008800F023
:108BF80027F800204A49087021E0ADB2002D09D1BC
:108C0800434800684670022000F01AF800204449E2
:108C1800087004E037003800C0B200F05CF80EE0DD
:108C2800ADB2002D04D037003800C0B200F053F8C0
:108C380005E0002000F004F8002039490870F1BD73
:108C480010B504003548006800280CD0210089B20E
:108C58002F480068314A1268904700202F49086061
:108C680000202549087010BD10B523480078002859
:108C780010D029480088FFF7E3FF2A48006850F021
:108C88000100284908602748006810F00100040026
:108C9800002CF8D110BD18B40200224B1B6833F029
:108CA8000403204C236000231800204B1B6813F09A
:108CB80001030093009B002B0BD0884209D2835CF0
:108CC8001B4C2360401C194B1B6813F001030093D5
:108CD800F0E712BC704710B5040006480068002889
:108CE80004D02000C0B203490968884710BD0000BD
:108CF8000860014078DC0020DBDC0020DADC0020A2
:108D080060DC0020D0DC002064DC002068DC00206F
:108D18006CDC0020D2DC0020D4DC002070DC0020D9
:108D2800DCDC00200060014074DC002004600140AD
:108D380010600140080421714B0000BA9E080548E4
:108D4800232E2B90B14E08EA3FB9E88BA9CAD60862
:108D580005D2E5BED127558208E5562A3B76769698
:108D68004808058E26D85D01A78808E289CC637972
:108D780095004B0805E075CDA4B946BC08EAD33781
:108D8800D29A8982EA08050CAE4CF5F63CB308E99C
:108D9800A770DFF1144F040805FE5BDF470A7C5B10
:108DA80008E2FB3E21A21BAA930805BFFDAB696C34
:108DB800A85A08E266B72E2C452DFB08050D55BDAF
:108DC800C237007208E2FF574D7C6C002C08059EE4
:108DD800F246FDD3161B08EA167F674DE5E2C80880
:108DE8000537331CFABBEEEF08EA005FBEA4FCBFF0
:108DF800C1080595122F0ACF558C08E770C2D4F028
:108E08008195C808E77200F98D1501A308E718E5F0
:108E18006C511F869F08E7DD37594BADB09C08E7BA
:108E2800C8E884CD55418308EF4F8E38CB37028789
:108E380008E7F500884C0965CE08EFDDBC6562AC33
:108E4800756208E7C0F15D98B0DD4308E719B4F82A
:108E58009F6D8CCB08E1DE63C232C6E42F0805F4AF
:108E680033B72E729AF908E765D938B8FE31160873
:108E7800E7F3062DF5FE0C3808E7704FE749B458BC
:108E88003908EFF146A9233864C008E7094E04D32E
:108E980046150208EF8DC720C390874D08EF00AB39
:108EA8007F2702C6A008E723A6A6A427117D08EFFE
:108EB800B3F19E6AB319AF08E7ABF515785E48F8C9
:108EC80008EF5BB12EAF2AFF1608E730625C827AA2
:108ED8003F8308EF91A7D31B6485BE08E74D8194B3
:108EE800E4AAE8DB08EFA0CC4A23A57E3608EF0CFD
:108EF800724CFB265AEC08EF0E42FAAF49A0A808BC
:108F0800E76D12DF2B0C615808EAB69BDE81B9FFCA
:108F1800FF080504EBD812D68DE008EC29664BDE75
:108F2800B7DE3608050D28B90A89311A070281010A
:108F3800018CBA800813141100001B0000051100F1
:108F48000100000511000103200511100104211082
:108F580011200C000B0007027100058CBA8000007C
:108F6800051120010C511011200C18010008038074
:108F780000B0100CE800441011200C24078FD50015
:108F88000002C008001200280711200330017CA04D
:108F98000511200135E01011200C38110F0F801A2F
:108FA800200000280CA4230911200545030099017D
:108FB80000081120044B06091040061120025094A5
:108FC8000A06112002540307051120015700091150
:108FD80020055B40040478201011210C00CCA1303E
:108FE800A021D1B9C9EA0512111011210C0C0A04EB
:108FF80015FC0300CCA130A021D11011210C18B907
:10900800C9EA0512110A0415FC030005112201031F
:109018001D0B112307002C0E0B040C73030C1140BD
:109028000800430900004EC520FE08320000000079
:1090380000000005175610CAF005171310CAF005EE
:1090480011000101000511000103200511010100B3
:1090580000081102040000000000051110010114AD
:109068000511120106401011200C000B0007061A0A
:1090780080058CBA800003051120010C27101120EF
:109088000C18018008038000302000E800A31011AC
:10909800200C24032699019200C200542380AB07B8
:1090A800112003300188800511200135E0101120BE
:1090B8000C38112424801A800000290C84230E11F6
:1090C800200A458F010001000A06321840061120C7
:1090D8000250940A06112002540307051120015773
:1090E80000091120055B40040878201011210C00AC
:1090F800CCA130A021D1B9C9EA0512111011210C57
:109108000C0A0415FC0300CCA130A021D1101121B8
:109118000C18B9C9EA0512110A0415FC0300051157
:109128002201031D0B112307002C0E0B040C7303E3
:109138000C1140080042093B134EC520FE000000F8
:109148000000000003836BF2F7703BE1F4F3501367
:109158001F979AC71C14F135E8E7A126EB64CAD417
:10916800CF58D98ACCDBB2783828E26B3BAB8999E7
:10917800D0CF434DD34C28BF27BF78AC243C135ED7
:109188006FC75E106C4435E298B765F19B340E03E7
:109198007050C4D773D3AF258720FF3684A394C4F7
:1091A800A09F879AA31CEC6857EFBC7B546CD789A7
:1091B800BF081D5DBC8B76AF487826BC4BFB4D4E77
:1091C800DE8EBD20DD0DD6D229FE86C12A7DED3387
:1091D800C11927E7C29A4C1536691C0635EA77F497
:1091E80011D664AA12550F58E6A65F4BE52534B987
:1091F8000E41FE6D0DC2959FF931C58CFAB2AE7E57
:10920800B149E330B2CA88C24639D8D145BAB32386
:10921800AEDE79F7AD5D120559AE42165A2D29E436
:109228007E113ABA7D9251488961015B8AE26AA946
:109238006186A07D6205CB8F96F69B9C9575F06E36
:10924800BC1D7B41BF9E10B34B6D40A048EE2B5216
:10925800A38AE186A0098A7454FADA675779B19526
:109268007345A2CB70C6C9398435992A87B6F2D816
:109278006CD2380C6F5153FE9BA203ED9821681FE6
:10928800D3DA2551D0594EA324AA1EB027297542F6
:10929800CC4DBF96CFCED4643B3D847738BEEF85A6
:1092A8001C82FCDB1F019729EBF2C73AE871ACC8B6
:1092B8000315661C00960DEEF4655DFDF7E6360FA6
:1092C8006293C6616110AD9395E3FD8096609672D6
:1092D8007D045CA67E8737548A74674789F70CB586
:1092E800ADCB1FEBAE4874195ABB240A59384FF856
:1092F800B25C852CB1DFEEDE452CBECD46AFD53F46
:109308000D5498710ED7F383FA24A390F9A7C86275
:1093180012C302B611406944E5B33957E63052A585
:10932800C20C41FBC18F2A09357C7A1A36FF11E835
:10933800DD9BDB3CDE18B0CE2AEBE0DD29688B2F05
:10934800783BF6827BB89D708F4BCD638CC8A69115
:1093580067AC6C45642F07B790DC57A4935F3C5605
:10936800B7632F08B4E044FA401314E943907F1B15
:10937800A8F4B5CFAB77DE3D5F848E2E5C07E5DCC5
:1093880017FCA892147FC360E08C9373E30FF881F5
:10939800086B32550BE859A7FF1B09B4FC986246C5
:1093A800D8A47118DB271AEA2FD44AF92C57210BB5
:1093B800C733EBDFC4B0802D3043D03E33C0BBCCC5
:1093C800A6B54BA2A536205051C5704352461BB1D5
:1093D800B922D165BAA1BA974E52EA844DD18176A5
:1093E80069ED92286A6EF9DA9E9DA9C99D1EC23B55
:1093F800767A08EF75F9631D810A330E828958FC65
:10940800C97215B2CAF17E403E022E533D8145A174
:10941800D6E58F75D566E4872195B4942216DF6664
:10942800062ACC3805A9A7CAF15AF7D9F2D99C2B34
:1094380019BD56FF1A3E3D0DEECD6D1EED4E06ECE4
:10944800C4268DC3C7A5E6313356B62230D5DDD044
:10945800DBB11704D8327CF62CC12CE52F42471714
:109468000B7E544908FD3FBBFC0E6FA8FF8D045AC4
:1094780014E9CE8E176AA57CE399F56FE01A9E9DD4
:10948800ABE1D3D3A862B8215C91E8325F1283C004
:10949800B4764914B7F522E6430672F540851907F4
:1094A80064B90A59673A61AB93C931B8904A5A4AC4
:1094B8007B2E909E78ADFB6C8C5EAB7F8FDDC08D74
:1094C8001AA830E3192B5B11EDD80B02EE5B60F0A4
:1094D800053FAA2406BCC1D6F24F91C5F1CCFA3794
:1094E800D5F0E969D673829B2280D2882103B97AA4
:1094F800CA6773AEC9E4185C3D17484F3E9423BD54
:10950800756F6EF376EC0501821F5512819C3EE063
:109518006AF8F434697B9FC69D88CFD59E0BA42733
:10952800BA37B779B9B4DC8B4D478C984EC4E76A23
:10953800A5A02DBEA623464C52D0165F51537DAD33
:10954800080421714B0000BA9E080548232E2B9071
:10955800B14E08EA3FB9E88BA9CAD60805D2E5BEDC
:10956800D127558208E5562A3B7676964808058E17
:1095780026D85D01A78808E289CC637995004B0855
:1095880005E075CDA4B946BC08EAD337D29A8982DA
:10959800EA08050CAE4CF5F63CB308E9A770DFF114
:1095A800144F040805FE5BDF470A7C5B08E2FB3EBC
:1095B80021A21BAA930805BFFDAB696CA85A08E253
:1095C80066B72E2C452DFB08050D55BDC237007218
:1095D80008E2FF574D7C6C002C08059EF246FDD32F
:1095E800161B08EA167F674DE5E2C8080537331CE5
:1095F800FABBEEEF08EA005FBEA4FCBFC108059500
:10960800122F0ACF558C08E770C2D4F08195C8088C
:10961800E77200F98D1501A308E718E56C511F865C
:109628009F08E7DD37594BADB09C08E7C8E884CD03
:1096380055418308EF4F8E38CB37028708E7F5008E
:10964800884C0965CE08EFDDBC6562AC756208E739
:10965800C0F15D98B0DD4308E719B4F89F6D8CCB75
:1096680008E1DE63C232C6E42F0805F433B72E7270
:109678009AF908E765D938B8FE311608E7F3062DD8
:10968800F5FE0C3808E7704FE749B4583908EFF190
:1096980046A9233864C008E7094E04D346150208D2
:1096A800EF8DC720C390874D08EF00AB7F2702C618
:1096B800A008E723A6A6A427117D08EFB3F19E6AA8
:1096C800B319AF08E7ABF515785E48F808EF5BB15A
:1096D8002EAF2AFF1608E730625C827A3F8308EFD4
:1096E80091A7D31B6485BE08E74D8194E4AAE8DB03
:1096F80008EFA0CC4A23A57E3608EF0C724CFB2657
:109708005AEC08EF0E42FAAF49A0A808E76D12DF3D
:109718002B0C615808EAB69BDE81B9FFFF080504E7
:10972800EBD812D68DE008EC29664BDEB7DE36089A
:10973800050D28B90A89311A07028101018CBA80FE
:1097480008131310000000000006110002000000BA
:109758000511000103200511010100000811020490
:1097680000000000000511100104211011200C0058
:109778000B00070C3500058CBA800001051120018B
:109788000C931011200C1801800803800030200071
:10979800E800511011200C24064D32032900C200A4
:1097A800542380AA071120033001AC800511200141
:1097B80035E01011200C38111212801A20000028F0
:1097C8000C842309112005458F0080010005112014
:1097D800014B06061120024D184006112002509434
:1097E8000A06112002540307051120015700091128
:1097F80020055B40040478201011210C007E641BB6
:10980800BA580BDDCED6E6F6001011210C0C030376
:1098180015F03F007E641BBA580B1011210C18DD9F
:10982800CED6E6F600030315F03F00081122040027
:109838000805001D0B112307002C0E0B040C7303E5
:109848000C1140080042093B13064D20FE000000A1
:1098580080B570480078002819D16F48F9F7F8FFEB
:1098680000211420FEF76AFC6C48006830F40050B0
:109878006A4908606948006850F400406749086010
:1098880001206449087066480068F8F7B1FD01BD19
:1098980080B560480078002824D05FF04050006808
:1098A80080061FD45FF040500068C0071AD45FF0EC
:1098B80040500068800715D40120F8F799FD5748F3
:1098C800006850F40050554908605448006830F466
:1098D80000405249086000211420FEF742FC002095
:1098E8004C49087001BD10B55FF040500468E007AE
:1098F80028D44C4801684C48FDF726FE01204B4906
:1099080008804A48807810F00F0050F0500047490E
:1099180088704648807810F0F000444988703822F2
:1099280043494248FEF778FE5FF04050006850F027
:1099380001005FF0405108603E480088401C3D49E6
:1099480008802DE0A00728D4364801683648FDF77E
:10995800FBFD0120354908803448807810F00F005D
:1099680050F05000314988703048807810F0F0008D
:109978002E498870382230492C48FEF74DFE5FF09A
:109988004050006850F002005FF0405108602948DC
:109998000088401C2749088002E02848F9F758FF4A
:1099A80010BD38B504001B480078002801D1FDF728
:1099B800F9FD23480068F8F71BFD1A480068FDF711
:1099C800DFFD050015F1010F03D100201D490870C6
:1099D8001DE0002D13D11B4800781B4909688842F7
:1099E80007DBFFF735FFFFF77EFF002015490870FA
:1099F800D9E714480078401C1249087007E0FFF7BF
:109A080027FFFFF770FF00200E490870CBE7FFF72C
:109A18003FFFC8E7DFDC002060B500008830014068
:109A2800E0B50000E4B5000037D7002034D70020A7
:109A38000020003064DB00200040003008B5000042
:109A4800E8B50000E0DC0020ECB50000816807E024
:109A580002681168536889185B18C360083202608D
:109A6800C2689142F4D04A1C8260087870472DE998
:109A7800FF4D00F10801009100270268520801EB30
:109A8800C2010191B8460021029103910168490879
:109A980000EBC101406800F0010501F1080440082D
:109AA80004EBC00630E000A8FFF7D0FF4FFA80FAB9
:109AB8000AE0009801680818009902904968081897
:109AC8000390009808300090029803998842F0D0DB
:109AD80010F801BB029047450CD1B44208BF00F012
:109AE8001DF8276805B14F44606800EB0708083483
:109AF8004745F2D0BAF1000F07F801BB0AD51AF1B1
:109B0800010AE8D14745CED1B442CCD1304604B0A1
:109B1800BDE8F08DBAF1010AD6D5F3E7012000F0CF
:109B280001B800002021090326311820ABBEF9E74F
:109B3800010000200322114202D0002210002CE074
:109B48000C22114202D00122100026E030221142DC
:109B580002D00222100020E0C022114202D00322CB
:109B680010001AE04FF44072114202D00422100093
:109B780013E04FF44062114202D0052210000CE0BD
:109B88004FF44052114202D00622100005E04FF473
:109B98004042114201D00722100040B2704730B550
:109BA80085B000A812491022F8F7F0FA0F480068AB
:109BB8000500280080B2FFF7BBFF040000A864B2CC
:109BC80030F814008543084864B250F8240000288F
:109BD80004D0054864B250F824008047ADB2002D87
:109BE800E7D105B030BD00000CDB00200430004098
:109BF800F8B40000012110F01F029140264A40B23B
:109C0800430942F82310704780B52220FFF7F2FF7E
:109C180001BD10B504005FF040500068400717D53B
:109C280007221E491E48FEF7F7FC002319221D498A
:109C38001D48FDF723FD5FF04050006830F0040038
:109C48005FF04051086019484088401C1749488017
:109C58005FF040500068000717D507220F491448E5
:109C6800FEF7DAFC002319220E490F48FDF706FD1E
:109C78005FF04050006830F008005FF04051086025
:109C88000A484088401C094948800A20F8F7B0FB78
:109C9800012008490870BEE780E200E048DB0020A8
:109CA800006000304BDB0020D0DA002064DB0020AD
:109CB80000800030DEDC002070B41F4803001F481D
:109CC8001F4D28601F480400B4F1204F08D9002018
:109CD8001D4D286000201D4D286001201C4D286066
:109CE80000201C4D2860FF201B4D28601B48006881
:109CF80010F0030001001A48006810F01C00020070
:109D0800002901D1142A0AD1164E3000164E35000A
:109D1800A84204D25FF0CD360660001DF8E70120A6
:109D280070BC70470020114908601148006850F065
:109D380020000F4908607047000000000000000084
:109D480008ED00E000000020008003401080034080
:109D5800088003403080034034800340388003404B
:109D6800180802404009002040090020400902402C
:109D780094810340000000002648006800F00300BA
:109D8800002804D021482249234A00F004F8234837
:109D9800804723480047884237D000F00306002E4A
:109DA80014D04FF00405A5EB06044FF0080707FB95
:109DB80006F8914669FA08F9002C07D080F8009057
:109DC80069FA07F900F10100641EF5E74FF0000693
:109DD8000F46091A88460911914614461546B1429C
:109DE80006D018BFA0E8340206F10106B142F8D146
:109DF80008F00F08B8F1000F07D002704FEA3222BE
:109E080000F10100B8F10108F4E7704740010020B3
:109E1800400900203880034000000000856F0000E2
:109E28006DB50000FEE7FEE7FEE7FEE7FEE7FEE7AA
:109E3800FEE7FEE7FEE7FEE7FEE7FEE7FEE7FEE7F2
:109E4800FEE7FEE7FEE7FEE7FEE7FEE7FEE7FEE7E2
:109E5800FEE7FEE7FEE7FEE7FEE7FEE7FEE7FEE7D2
:109E6800FEE7FEE7FEE7FEE7FEE7FEE7FEE7FEE7C2
:109E7800FEE7FEE7FEE7FEE7FEE7FEE7FEE7FEE7B2
:109E8800FEE7FEE7FEE7FEE7FEE7FEE7FEE7FEE7A2
:109E9800FEE7FEE7FEE7FEE7FEE7FEE7FEE7FEE792
:109EA800FEE7FEE7FEE7FEE7FEE7FEE7FEE7FEE782
:109EB800FEE7FEE7FEE7FEE7FEE7FEE7FEE7FEE772
:109EC800FEE7FEE700300140043001400830014061
:109ED8000C3001401030014014300140183001406E
:109EE8001C3001402030014024300140283001401E
:109EF8002C300140303001403430014038300140CE
:109F08003C3001404030014044300140483001407D
:109F18004C3001405030014054300140583001402D
:109F28005C300140603001406430014068300140DD
:109F38006C3001407030014074300140783001408D
:109F48007C300140417474656D707420746F2073A7
:109F5800656E64205854454120656E63727970744B
:109F68006564207061636B65742C2062757420438E
:109F780053502077617320636F6D70696C6564203E
:109F8800776974686F7574205854454120737570EB
:109F9800706F72742E2044697363617264696E67AE
:109FA800207061636B6574005244503A20526563B7
:109FB800656976656420696E20532025753A20739B
:109FC800796E2025752C2061636B2025752C206502
:109FD80061636B2025752C207273742025752C20E5
:109FE8007365715F6E72202535752C2061636B5F18
:109FF8006E72202535752C207061636B65745F6CFB
:10A00800656E202575202825752900004174746522
:10A018006D707420746F2073656E64207061636B5B
:10A028006574207769746820484D41432C20627517
:10A0380074204353502077617320636F6D70696C8F
:10A04800656420776974686F757420484D414320B2
:10A05800737570706F72742E2044697363617264D3
:10A06800696E67207061636B657400005265636593
:10A0780069766564205854454120656E637279702D
:10A08800746564207061636B65742C20627574203C
:10A098004353502077617320636F6D70696C6564FA
:10A0A80020776974686F757420585445412073751A
:10A0B80070706F72742E2044697363617264696E84
:10A0C80067207061636B65740000000041747465FB
:10A0D8006D707420746F2063726561746520736F8E
:10A0E800636B657420746861742072657175697238
:10A0F800657320585445412C206275742043535091
:10A108002077617320636F6D70696C65642077696F
:10A1180074686F7574205854454120737570706F5A
:10A1280072740000417474656D707420746F2063DC
:10A13800726561746520736F636B65742074686100
:10A148007420726571756972657320484D41432C9E
:10A1580020627574204353502077617320636F6DBC
:10A1680070696C656420776974686F757420484DF0
:10A17800414320737570706F727400004174746588
:10A188006D707420746F2063726561746520484D2A
:10A1980041432061757468656E74696361746564B0
:10A1A800207061636B65742C206275742043535072
:10A1B8002077617320636F6D70696C6564207769BF
:10A1C80074686F757420484D414320737570706FC3
:10A1D8007274000052656365697665642070616316
:10A1E8006B6574207769746820484D41432C206260
:10A1F8007574204353502077617320636F6D7069C5
:10A208006C656420776974686F757420484D4143A4
:10A2180020737570706F72742E2044697363617255
:10A2280064696E67207061636B657400417474655E
:10A238006D707420746F2063726561746520585462
:10A24800454120656E63727970746564207061633E
:10A258006B65742C206275742043535020776173AA
:10A2680020636F6D70696C656420776974686F75B9
:10A2780074205854454120737570706F72740000D3
:10A2880070B504000D00160010480068002809D1B8
:10A2980003225FF4E1310E480068FCF754FC01200A
:10A2A8000A490860002D01D100200DE0012C04D0DE
:10A2B800022C02D05FF0FF3006E03200290004488B
:10A2C8000068FCF75DFC300070BD00BFCCDC0020EE
:10A2D800F0B500004F6E6C7920706F727473206651
:10A2E800726F6D20302D25752028616E64204353D0
:10A2F800505F414E5920666F722064656661756CC7
:10A3080074292061726520617661696C61626C658F
:10A3180020666F7220696E636F6D696E6720706F5B
:10A32800727473004C657373207468616E206F6E6D
:10A33800652077696E646F77206672656520696E3F
:10A348002052585F71756575652C20646566657265
:10A3580072696E672061636B6E6F776C6564676D99
:10A36800656E7420666F7220256875004F55543AE3
:10A3780020532025752C20442025752C204470203E
:10A3880025752C2053702025752C2050722025759A
:10A398002C20466C203078253032582C20537A20D7
:10A3A8002575205649413A20257300005253542000
:10A3B800726563656976656420696E20434C4F5306
:10A3C800455F57414954206F7220434C4F534544D1
:10A3D8002E204E6F7720636C6F73696E6720636FF2
:10A3E8006E6E656374696F6E00000000494E503AE6
:10A3F80020532025752C20442025752C20447020BE
:10A4080025752C2053702025752C20507220257519
:10A418002C20466C203078253032582C20537A2056
:10A42800256875205649413A2025730019E050F8EF
:10A43800041BCB0744BFA9F101035918121F0023BD
:10A44800042A41F8043BF9D25FEA827C0B4604D522
:10A458004FF0000CA1F800C09B1CD10744BF00219D
:10A46800197050F8042B002AE1D170475245534522
:10A478005420696E2073657175656E63652C206E56
:10A488006F206D6F7265206461746120696E636FFF
:10A498006D696E672C207265706C792077697468B5
:10A4A80020524553455400005244503A2044656CAC
:10A4B800617965642061636B733A2025752C20618E
:10A4C800636B2074696D656F75742025752C206128
:10A4D800636B2065616368202575207061636B6517
:10A4E80074000000417474656D707420746F20638B
:10A4F800726561746520524450207061636B6574A5
:10A50800206F6E20636F6E6E656374696F6E2D6C5D
:10A5180065737320736F636B657400005244503A1F
:10A528002057696E646F772053697A652025752CEA
:10A5380020636F6E6E2074696D656F757420257564
:10A548002C207061636B65742074696D656F757418
:10A5580020257500496E76616C6964207365717594
:10A56800656E6365206E756D62657221202568755C
:10A57800206E6F74206265747765656E2025687536
:10A5880020616E64202568750000000052656365CF
:10A5980069766564207061636B6574207769746897
:10A5A8006F757420524450206865616465722E206E
:10A5B80044697363617264696E67207061636B6577
:10A5C8007400000070B504000D001600F7F77AF863
:10A5D800D5F80A10C1F30451C9B2C0B2814204D0FF
:10A5E8002800F6F7F6FE002005E0002202492800C0
:10A5F800F8F7EAFF002070BD440000204661696C4E
:10A60800656420746F206372656174652071756577
:10A6180075657320666F722052445020696E2063FE
:10A6280073705F636F6E6E5F696E6974000000001F
:10A638004552524F523A20526F7574696E672069BD
:10A648006E707574204649464F2069732046554CF4
:10A658004C2E2044726F7070696E67207061636B56
:10A6680065742E004E6F742053594E2072656365D1
:10A678006976656420696E20434C4F5345442073C6
:10A68800746174652E2044697363617264696E67CE
:10A69800207061636B6574004661696C6564207441
:10A6A8006F20696E697469616C697A652043414EEF
:10A6B800206964656E74696669636174696F6E2088
:10A6C8006E756D626572000043616E6E6F74206412
:10A6D8006571756575652066726F6D2072785F713A
:10A6E8007565756520696E20717565756520646589
:10A6F8006C6976657200000043616E6E6F74206449
:10A708006571756575652066726F6D2072785F7109
:10A718007565756520696E20717565756520657844
:10A72800697374730000000043616E6E6F74206477
:10A738006571756575652066726F6D2074785F71D7
:10A748007565756520696E20636865636B2074693B
:10A758006D656F7574000000496E76616C696420E0
:10A7680041434B206E756D62657221202575206E00
:10A778006F74206265747765656E20257520616E3B
:10A78800642025750000000052656365697665647C
:10A79800207061636B657420776974686F757420C5
:10A7A80043524333322E20416363657074696E6788
:10A7B800207061636B6574004661696C6564207420
:10A7C8006F206765742062756666657220666F72B1
:10A7D800204353505F424547494E207061636B6583
:10A7E800740000006373705F6E6577207061636B3F
:10A7F80065742063616C6C65642077697468204EA9
:10A80800554C4C20696E7465726661636500000082
:10A818004552524F5220736F636B65742063616EAB
:10A828006E6F7420616363657074206D6F7265204C
:10A83800636F6E6E656374696F6E73005258205152
:10A84800756575652064656C69766572206D6174DF
:10A858006368696E6720456C656D656E742C20733E
:10A868006571202575000000525820517565756581
:10A8780020657869737473206D61746368696E67A5
:10A8880020456C656D656E742C2073657120257587
:10A898000000000043616E6E6F7420646571756519
:10A8A80075652066726F6D2074785F717565756562
:10A8B80020696E20666C757368204541434B000023
:10A8C800545820456C656D656E7420467265652C1C
:10A8D8002074696D652025752C2073657120257598
:10A8E8002C20756E61202575000000005458204505
:10A8F8006C656D656E742074696D6564206F757420
:10A908002C2072657472616E736D697474696E67F8
:10A9180020736571202575005245534554206F7585
:10A9280074206F662073657175656E63652C206B86
:10A9380065657020636F6E6E656374696F6E206FF6
:10A9480070656E00435243333220766572696669DA
:10A95800636174696F6E206572726F722120446939
:10A968007363617264696E67207061636B657400FC
:10A97800417474656D707420746F20616C6C6F63C2
:10A9880061746520746F6F206C6172676520626CFA
:10A998006F636B2025750000465245453A20556E79
:10A9A800616C69676E656420435350206275666602
:10A9B800657220706F696E746572202570000000E2
:10A9C800436F756C64206E6F7420696E6974696179
:10A9D8006C697A65204346502069642073656D610F
:10A9E80070686F72650000004661696C6564207468
:10A9F8006F2067657420434650206964656E7469EA
:10AA08006669636174696F6E206E756D6265720048
:10AA18004661696C656420746F2073656E642043B9
:10AA2800414E206672616D6520696E206373705FA8
:10AA380074785F63616E00004661696C65642074B8
:10AA48006F2073656E642043414E206672616D65A8
:10AA580020696E2054782063616C6C6261636B00BE
:10AA68004661696C656420746F20696E69746961F8
:10AA78006C697A652043414E207061636B65742070
:10AA880062756666657273004B49535320696E762A
:10AA9800616C696420637263206672616D652073FE
:10AAA8006B69707065642C206C656E3A20257500A2
:10AAB8006373705F73656E645F6469726563742045
:10AAC80063616C6C65642077697468204E554C4CE2
:10AAD800207061636B6574006373705F6E657720C7
:10AAE8007061636B65742063616C6C656420776961
:10AAF8007468204E554C4C207061636B657400007F
:10AB0800494E54455246414345204552524F523AC8
:10AB1800206E6F7420706F737369626C6520746F38
:10AB28002073656E640000004541434B20636F6DE0
:10AB38007061726520656C656D656E742C20746932
:10AB48006D652025752C2073657120257500000022
:10AB58004E756C6C20706F696E74657220706173CD
:10AB680073656420746F2072647020666C757368F6
:10AB780020616C6C00000000466F756E64206120D7
:10AB88006C6F737420636F6E6E656374696F6E2C7F
:10AB980020636C6F73696E67206E6F77000000002A
:10ABA80048616C662D6F70656E20636F6E6E6563AD
:10ABB80074696F6E20666F756E642C2073656E64A1
:10ABC800696E6720525354005244503A20437265CC
:10ABD8006174696E6720524450207175657565739C
:10ABE80020666F7220636F6E6E2025700000000073
:10ABF80052445020436C6F736520696E20434C4F5C
:10AC080053455F574149542C206E6F7720636C6F12
:10AC180073696E67000000004661696C65642074A2
:10AC28006F2073657420726F7574653A20696E764B
:10AC3800616C6964206E6F64652069642025750005
:10AC48005761726E696E6720736F636B65742063FA
:10AC58006F6E6E656374696F6E20717565756520BA
:10AC680066756C6C0000000010B5044614F1010F05
:10AC780082B00AD08DF80000012200A90120FFF758
:10AC8800FFFA012801D1204616BD4FF0FF3016BD4E
:10AC980010B5074979441831064C7C44163404E051
:10ACA8000A68081D511888470146A142F8D110BD0D
:10ACB8002402000068020000465245453A20496EC9
:10ACC80076616C69642043535020627566666572CC
:10ACD80020706F696E746572202570004652454574
:10ACE8003A2042756666657220257020696E207567
:10ACF800736520627920257520757365727300006D
:10AD08004E6F206D6F7265206D656D6F727920666C
:10AD18006F722073706F72742073656D6170686FE5
:10AD2800726500004661696C656420746F20637207
:10AD38006561746520636F6E6E656374696F6E20FC
:10AD48006C6F636B000000004E6F206D6F726520A2
:10AD58006D656D6F727920666F7220636F6E6E20FD
:10AD680073656D6170686F72650000004E6F2061D9
:10AD78007661696C61626C65207061636B657420D3
:10AD880062756666657220666F722043414E0000E8
:10AD98004F7574206F66206F72646572204D4F5234
:10ADA80045206672616D65207265636569766564C4
:10ADB80000000000526563656976656420756E6BF6
:10ADC8006E6F776E20434650206D657373616765BB
:10ADD80020747970650000004B4953532073686FE5
:10ADE8007274206672616D6520736B69707065643A
:10ADF8002C206C656E3A202575000000466C757332
:10AE08006820545820456C656D656E742C207469F3
:10AE18006D652025752C207365712025750000004F
:10AE2800466C75736820525820456C656D656E7464
:10AE38002C2074696D652025752C2073657120257B
:10AE480075000000496E76616C69642053594E2084
:10AE58006F72206E6F2041434B2C207265736574AE
:10AE680074696E6721000000496E76616C69642020
:10AE780053594E206F72206E6F2041434B20696EEC
:10AE880020434C4F53452D57414954004661696C46
:10AE9800656420746F20637265617465205458205E
:10AEA800717565756520666F7220636F6E6E000040
:10AEB8004661696C656420746F20637265617465AE
:10AEC80020525820717565756520666F7220636F12
:10AED8006E6E000059F5FFFF18D30000CC09002062
:10AEE800000000008BEBFFFF0200000002000000E2
:10AEF800FC060000D6000000000000203C01000015
:10AF08006FEBFFFF0200000002000000B607000020
:10AF180008000000400900208C000000417474659E
:10AF28006D707420746F2066726565206E756C6C28
:10AF380020706F696E7465720000000046524545C6
:10AF48003A2042756666657220616C726561647943
:10AF58002066726565202570000000005258207137
:10AF6800756575652025702066756C6C2077697429
:10AF780068202575206974656D7300004E554C4C2A
:10AF880020506F696E74657220676976656E2074EB
:10AF98006F206373705F636C6F73650043414E206D
:10AFA80042756666657220656C656D656E742074A1
:10AFB800696D6564206F75740000000043414E2080
:10AFC8006672616D65206C6F737420696E204353DF
:10AFD80050207061636B6574000000004661696C05
:10AFE800656420746F206372656174652043414E07
:10AFF8002052582071756575650000004661696CBE
:10B00800656420746F20696E697469616C697A651A
:10B018002043414E206472697665720042696E640D
:10B02800696E6720736F636B657420257020746F79
:10B0380020706F727420257500000000496E7661DB
:10B048006C6964207265706C7920746F2053594E56
:10B0580020726571756573740000000049676E6F32
:10B0680072696E67206475706C69636174652053DA
:10B07800594E207061636B657421000057616974D3
:10B08800696E6720666F722075736572737061638D
:10B098006520746F20636C6F736500004661696C8E
:10B0A800656420746F20696E697469616C697A657A
:10B0B8002073656D6170686F72650000524450209E
:10B0C800436C6F73652C2073656E74205253542043
:10B0D8006F6E20636F6E6E2025700000546F6F20B6
:10B0E80073686F7274207061636B657420666F7229
:10B0F8002043524333322C20257500004E6F206DBB
:10B108006F726520636F6E6E656374696F6E73200E
:10B11800617661696C61626C65000000436F6E6EF8
:10B12800656374696F6E20627566666572207175F5
:10B138006575652066756C6C210000003233343506
:10B14800363738393A3B3C3D3E3F4041424344451F
:10B15800464748494A4B4C4D4E4F50514661696CE1
:10B16800656420746F206C6F636B20636F6E6E2054
:10B1780061727261790000004E6F206D6F726520F8
:10B188006672656520636F6E6E656374696F6E7352
:10B198000000000053686F727420424547494E20F2
:10B1A8006672616D65207265636569766564000025
:10B1B8004661696C656420746F20696E6974204308
:10B1C800414E205258207461736B0000506F7274A6
:10B1D80020256420697320616C7265616479206937
:10B1E8006E207573650000005244503A204E503A64
:10B1F80020436F6E6E656374696F6E204F50454EC5
:10B208000000000053594E2D524356443A205772BD
:10B218006F6E672041434B206E756D62657200004A
:10B228005244503A204E433A20436F6E6E65637421
:10B23800696F6E204F50454E000000004475706CD9
:10B2480069636174652073657175656E6365206EE9
:10B25800756D6265720000005244503A20455252A2
:10B268004F522064656661756C74207374617465EF
:10B2780021000000436F6E6E2D6C65737320736F31
:10B28800636B65742071756575652066756C6C00F7
:10B298004661696C656420746F20737461727420F0
:10B2A800726F75746572207461736B00FEF704FD2C
:10B2B800002801D0FFF7ECFC0020FEF733FDFCF777
:10B2C800B0F800F000F800F001B800000746384672
:10B2D800FEF728FCFBE700004C6576656C202575B9
:10B2E8003A2076616C75652025750D0A000000000E
:10B2F800496E76616C696420736F636B6574206F47
:10B308007074696F6E0000004E6F20726F757465FF
:10B3180020746F20686F73743A20252330387800C2
:10B32800435243333220617070656E6420666169F0
:10B338006C6564210000000052657472616E736D63
:10B34800697373696F6E206661696C6564000000DB
:10B35800476F7420524553455420696E20737461B9
:10B368007465202575000000526F7574657220663B
:10B3780061696C656420746F2073656E64000000F9
:10B3880038B504460D462846FFF76EFCA84218BF9C
:10B398000024204632BD0000436F7272757074201D
:10B3A800435350206275666665720000436F6E6E87
:10B3B80020616C726561647920636C6F73656400E9
:10B3C8004D6178206C6576656C20697320360D0AAE
:10B3D80000000000496E636F6D706C6574652066CF
:10B3E80072616D65000000005258206275666665DE
:10B3F80072206F766572666C6F770000556E6B6EA3
:10B408006F776E2043414E206D6F64650000000029
:10B418004B495353205258206F766572666C6F778C
:10B42800000000004164646564204541434B206E80
:10B438007220257500000000436F6E6E2052582060
:10B448006275666665722066756C6C005458204596
:10B458006C656D656E74202575206672656564007F
:10B46800434C4F53455F574149542074696D656F8C
:10B47800757400005244503A2053594E2D5265635A
:10B48800656976656400000046726565204D656DE6
:10B498006F72793A2025640A0000000046726565DB
:10B4A800204D696E696D69616C3A2025640A000057
:10B4B8004F7574206F66206275666665727300004A
:10B4C80044656C6976657220736571202575000086
:10B4D800576520686176652061206D617463680036
:10B4E800727373692069732025640D0A0A000000CD
:10B4F80003000C003000C0000003000C003000C046
:10B50800616C6C20747820627573790A0000000001
:10B518004745543A2025702025700000465245457D
:10B528003A20257000000000576169743A202570A0
:10B5380000000000506F73743A202570000000006E
:10B548001B5B25753B25756D0000000057446F6730
:10B558002066656564210A007374617274207478CA
:10B568000A000000C046C046C046C046FFF79EFE1F
:10B578004C4F4F50000000004B495353000000004F
:10B5880052465F525800000052465F54580000006F
:10B59800424541434F4E00000001000102020303EF
:10B5A80049444C450000000043414E001300000090
:10B5B8000000000013000000000000000700000069
:10B5C80008000000000000000800000043414E0091
:10B5D80007000000F0E300E001000000DC000000CC
:10B5E800010000000A00000050DA0020010101FA01
:10B5F8000001B0B5FA0001355BFD000001D2000181
:10B6080078B5FA0001CDA5CE000810270000E803A0
:10B61800000001FD0002200401FB003FD4B500003A
:10B62800B9C3CBD1D4D8DADCDEE0E2E3E5E6E7E87B
:10B63800EAEBECEDEEEEEFF0F1F2F2F3F4F5F5F6FD
:10B64800F7F7F8F9F9FAFAFBFBFCFDFDFEFEFFFF40
:10B65800000001010202030304040505FD060507B5
:10B668000708080909FD0A030B0B0C0CFD0D030E56
:10B678000E0F0FFD10011111FD120313131414FD09
:10B6880015011616FD170318181919FD1A051B1BA5
:10B698001C1C1D1DFD1E091F1F20202121222223E5
:10B6A80023FD00FCAA1B0024F4000024F40000245D
:10B6B800F4000024F4000024F4000024F400002422
:0AB6C800F400FC0000018100F8000E
:040000050000B56DD5
:00000001FF
